:1000000000000220F1710000197200001B72000054
:100010001D7200001F72000021720000000000002D
:10002000000000000000000000000000237200003B
:1000300025720000000000002772000029720000F5
:100040002B7200002D510000997600001D710000F8
:10005000297100002B7200002B7200002B7200002F
:100060002B7200002B7200001D3300002B72000069
:100070002B7200002B7200002B7200002B7200000C
:100080002B7200001D7700002B7200002B72000005
:100090002B7200002B7200002B7200002B720000EC
:1000A0002B7200002B7200002B7200002B720000DC
:1000B0002B7200002B720000000000000000000006
:1000C0002B7200002B7200002B7200002B720000BC
:1000D0002B7200002B7200002B7200000000000049
:1000E0000000000000000000000000000000000010
:1000F0000000000000000000000000000000000000
:1001000000000000000000000000000000000000EF
:1001100000000000000000000000000000000000DF
:1004000010B5054C237833B9044B13B10448AFF34E
:1004100000800123237010BD340200200000000082
:1004200018CB000008B5034B1BB103490348AFF3D9
:10043000008008BD000000003802002018CB00003A
:10044000154B002B08BF134B9D46A3F5803A0021A6
:100450008B460F461348144A121A09F0F9FB0F4B4A
:10046000002B00D098470E4B002B00D0984700205F
:10047000002104000D000D48002802D00C48AFF305
:10048000008009F09DFB2000290007F05DF909F0CC
:1004900071FB00BF00000800000002200000000007
:1004A0000000000034020020F88D01200000000050
:1004B0000000000010F0010310D104280CD90368DB
:1004C000C3F30F1343B1013B9B001A1DC1180979F7
:1004D00011B101339342F9D1184670470023FBE76D
:1004E000037883B11A0601D40130704703F0C003CA
:1004F000C02B08BF0130024610460132037803F0DA
:10050000C003802BF8D0704708B5002103780BB9E1
:10051000084608BDFFF7E4FF0131F7E738B50022D0
:1005200004460D46411C092003F004FA40B1630063
:10053000024643F0010342F8043F0023A34200DBDC
:1005400038BD55F8231042F8041F0133F6E701289F
:1005500038B504DC1C20BDE8384000F0F9BF0D6858
:10056000EA0701D41120F6E74868C30706D4042837
:1005700004D9036803F00F03042B01D00E20EAE72F
:1005800003F03CF86D10002D044603DDFFF7BCFFBF
:10059000A84206DA1220DEE72046FFF7A1FF013D60
:1005A0000446012DF8D120787F2808DDDF280ADCF9
:1005B0006378800100F4F86003F03F0318434000C3
:1005C00040F0010038BDEF280ADC637800039B018E
:1005D00080B203F47C630343A07800F03F00EDE7B2
:1005E000F72810DC637880041B0303F47C3300F4E9
:1005F000E0101843E37803F03F030343A078800141
:1006000000F47C60DAE74FF0FF30D8E7486838B58F
:10061000C3070D4606D4042804D9036803F00F026B
:10062000092A04D00B20BDE8384000F091BF44688F
:10063000C3F30F1364105A1EA2420BD8032194FB7C
:10064000F1F16429A8BF64210329ACBF5918D91C52
:1006500003F0ACF90368C3F30F13013B9C4208D2CB
:10066000A31C013464002A6840F8232044F00104EC
:100670004460002038BD01282DE9F84304DC1C202B
:10068000BDE8F84300F064BF02284E680CD08C68C7
:10069000E70709D56410012CB8BF0124F50705D57B
:1006A0004FF0FF30BDE8F8830124F7E7042EF7D9B7
:1006B00033680D6803F00F02042A23D1E80706D43B
:1006C000042D04D92B6803F00F03042B01D00E2056
:1006D000D6E73046FFF7EEFEA042E1DB304602F0FF
:1006E0008DFF0646284602F089FF013C014630197D
:1006F00009F07BFE0028D3D0801B0130400040F081
:100700000100CFE7092A38D177687F10BC42C7DCE7
:10071000E90729D4042D27D92B6803F00F03042BF4
:1007200022D1284602F06AFF804604F1010956F8FA
:100730002900854203D1640044F00100B2E7C207FA
:100740000ED404280CD9036803F00F03042B07D13F
:1007500002F054FF0146404609F00EFE0028EAD0A0
:10076000B9454C46E1DD9BE7631C56F82320AA42BD
:10077000E1D0BB421C46F7DD92E7032A90D1C3F3D8
:100780000F17C3F34173C3EB8707BC4288DCEB0749
:1007900028D4042D26D9286800F00F03032B17D185
:1007A000C0F30F13C0F3417005F10408C0EB8300E0
:1007B0003F1A013C40440336BC423FF771AF321947
:1007C0004346834219460FD315D10134600096E7A2
:1007D000042B07D1284602F011FF80462846FFF778
:1007E00069FEE5E70F204BE712F8015F09788D42BB
:1007F00003F10103E5D00134DEE708B502F0E2FEC3
:10080000400040F0010008BDC30711D404280FD9EF
:10081000026802F00F03032B0AD101F00303C3F1B6
:1008200004035B0703F0C04322F0C042134303609C
:10083000704701282DE9F0470546884604DC1C2056
:10084000BDE8F04700F084BE4C6814F0010701D108
:100850000D20F5E7022802D08B68DA07F8D5D8F822
:100860000060F30700F1A980042E40F2A6803268F0
:100870006410012C02F00F03B8BF0124092B28D10A
:100880007668022D4FEA660605D0D8F808305B106E
:100890009E42A8BF1E46351B0135012225EAE5759B
:1008A000A918092003F046F8074648B16D00034631
:1008B00045F00105D8F8002043F8045FA64202DAAB
:1008C0003846BDE8F087013452F8241043F8041F7D
:1008D000F4E7042B43D1304602F090FEFFF714FEFC
:1008E000022D824605D0D8F808305B109842A8BF88
:1008F0009A46A24504DA0020BDE8F04703F094B818
:10090000304602F07BFE0546A74222DB304602F06D
:1009100075FEA94606462846FFF7E2FD0134A245CA
:100920000546F8DAA0EB0905284603F07DF80746EE
:100930000028C5D002F062FE0446D8F8000002F09C
:100940005DFEA9EB060101442A46204609F05CF948
:10095000B6E72846FFF7C4FD01370546D4E7032B69
:100960002BD1C2F30F13022DC2F34172C2EB8302EB
:1009700005D0D8F808305B109A42A8BF1A46A242A8
:1009800006DA002211460320BDE8F04702F0D2BF8C
:10099000151B0423291D002291FBF3F1032002F013
:1009A000C9FF074600288BD001352946FFF72CFFE9
:1009B000E11C2A4631440430C8E7212040E70028E2
:1009C000F8B504DC1C20BDE8F84000F0C1BD0C689F
:1009D00014F001060FD0641024EAE474E11C002234
:1009E0008910032002F0A6FF054610B12146FFF74B
:1009F0000BFF2846F8BD042C01D80025F9E725682F
:100A000005F00F05042D19D12046FFF753FD32469E
:100A1000C11C074691FBF5F1032002F08BFF054650
:100A20000028E6D03946FFF7EFFE204602F0E6FD4B
:100A30003A460146281D09F0E7F8DAE7092DDCD12E
:100A400067687F100423F91C324691FBF3F1032001
:100A500002F070FF05460028CFD03946FFF7D4FEDC
:100A60000434BE42C5DA54F8043FDA0742BFAA197B
:100A7000A3F3480313710136F3E77F2902DC017009
:100A800001307047B1F5006F0CDA03468A1162F04D
:100A90003F0203F8022B01F03F0161F07F0141703A
:100AA00018467047B1F5803F0FDA0B1363F01F0350
:100AB0000370C1F3851301F03F0163F07F0361F020
:100AC0007F014370817003307047B1F5883F0DDAC4
:100AD000F0230370902343708B1101F03F0163F00A
:100AE0007F0361F07F018370C170043070470000A4
:100AF0000028F7B50F4603DC1C2000F029FD0CE0B0
:100B00000A6812F001000AD06C4651102046FFF727
:100B1000B4FF011B204602F08EFF044616E0042AB3
:100B20003BD9136803F00F03092B36D155681C49D4
:100B30006D100124AC420CDD02F076FF044628B1B2
:100B40003F6802F05BFD0126AE421DDD204603B08A
:100B5000F0BD013452F8243013F0010601D10D200C
:100B6000CBE75B107F2B09DDB3F5006F08DBB3F536
:100B7000803F07DB8B42D4BF042600263044D9E7F0
:100B80000226FBE70326F9E7013657F82610CB07C4
:100B9000E5D54910FFF771FFD6E72120ADE700BF8B
:100BA000FF0F010010B5044611F0010011D1042916
:100BB0000ED90B6803F00F03042B09D1084602F08D
:100BC0001DFD0146204609F0D7FBB0FA80F0400930
:100BD00010BD0020FCE700000128F8B50E4604DC3B
:100BE0001C20BDE8F84000F0B3BC4D6815F00107CB
:100BF00006D1042D04D92B6803F00F02092A01D075
:100C00000B20EEE76C6809681F486410C3F30F13EC
:100C1000A34298BF03F1FF34FFF7C4FF40B10123A3
:100C2000BC4201DA0020F8BD013745F82730F7E76C
:100C300031681648FFF7B6FF50B1002CF2D0631CA4
:100C40000122013C944045F8232014436C60E9E7FD
:100C50003368DA0701D40D20C3E75B10002B0DDDEC
:100C60009C420BDB05EB830305EB84029A4207D120
:100C70000123013C9C4053601C43E7E71220B0E78E
:100C8000996843F8041FF1E7F7B20000FBB20000D7
:100C9000002310B50B70C3070C4606D50E49421051
:100CA0002046BDE8104009F02BBB28B90B4920466F
:100CB000BDE8104009F044BB042801D10849F6E71B
:100CC00009D9036803F00F03042B04D102F096FC4A
:100CD00004490246E4E710BD30BD000000B3000047
:100CE00006B300000BB300002DE9F04301288FB0DC
:100CF00081460E4607DC1C2000F02AFC05462846EB
:100D00000FB0BDE8F0830B6813F0010440F0A18040
:100D1000042B40F2D5801B6803F00F03092B40D150
:100D2000274656F8273013F0010806D1042B04D9C2
:100D3000186800F00F00092801D02220DCE75B686A
:100D40000137B94504EB6304EBD10122A11802F08D
:100D5000F1FD054608B90025D1E7640044F001041F
:100D60004460424600F1080456F822104B680868B7
:100D70005B10C0F30F10984298BF00F1FF330431AD
:100D80000020834207DC013223EAE373BA4204EB1A
:100D90008304E9DBB3E751F804CF44F820C0013005
:100DA000EFE7032B40F08C80274656F8270010F021
:100DB0000108C2D10428C0D9036803F00F02032A36
:100DC00038D1C3F30F12C3F34173C3EB82031C4446
:100DD0000137B945E9D10423E11C002291FBF3F16D
:100DE000032002F0A7FD05460028B4D02146FFF7F6
:100DF0000BFD00F1040956F82840E10720D4042C2B
:100E00001ED9206800F00F03032B19D1C0F30F1374
:100E1000C0F34170C0EB830003344B46A3EB0902DF
:100E2000824211DB08F101080028A8BF8144B845BF
:100E3000E1DB64E7042A80D1FFF73CFB0444C7E709
:100E40002046FFF737FBE7E714F8012F03F8012BE3
:100E5000E4E700252C4656F82500C20732D40428C2
:100E600030D9036803F00F02042A32D1FFF722FBC6
:100E700004440135A945EED1204602F0D5FD0546D2
:100E800000283FF468AF041DB04606EB890958F806
:100E9000046BF30728D4042E26D9336803F00F021D
:100EA000042A34D13046FFF705FB0746304602F0EE
:100EB000A5FB3A460146204608F0A6FE3C4421E048
:100EC0002546C8E701A9FFF7E3FE01A809F05EFA8D
:100ED000CEE7032A7FF431AFC3F30F12C3F341739C
:100EE000C3EB82031C44C4E701A93046FFF7D0FEE0
:100EF00001A809F04BFA01A906460246204608F06F
:100F000083FE3444C145C2D100232370F7E6032A8F
:100F1000F8D1C3F30F17C3F34173C3EB87073A4606
:100F2000311DC8E72DE9F04F002891B0894607DC54
:100F30001C2000F00DFB0446204611B0BDE8F08FE8
:100F40000C6814F0010706D1042C04D9236803F0BF
:100F50000F03092B01D00B20EBE766687610002EFB
:100F600003DC384602F060FDE5E701286BD04868F5
:100F7000C50768D4042866D9036803F00F03042B5F
:100F800061D102F03BFB0546284609F0FFF9043425
:100F900006F1FF3A04EB860380460AFB00FB009350
:100FA00054F8040FC10750D404284ED9026802F047
:100FB0000F02042A50D1FFF77DFA009BA34283441D
:100FC000EED1584602F030FD04460028B4D0D9F8DE
:100FD00000B0B8F1000F04D0D9F8040002F00EFB05
:100FE0000546204602F00AFB0BF1040B81465BF834
:100FF000043F0093184602F001FB009BDA0701460C
:1010000001D4042B04D803A91846FFF741FE03A915
:101010000846019109F0BAF9019900900246484644
:1010200008F0F2FD009B9944B8F1000F07D0BA45D3
:1010300005DD48464246294608F0E6FDC144013731
:10104000BE42D4D178E7064D9EE703A9FFF720FE04
:1010500003A809F09BF9B0E702F0D0FAF9E700BF66
:101060009FB70000002810B511DD0B6813F00104D4
:1010700002D05C1024EAE4740122A118092002F0D5
:1010800059FC18B1640044F00104446010BD002410
:10109000F2E70A6838B512F0010436D1042A34D9CF
:1010A0001368496803F00F00092818D15068C3F38A
:1010B0000F134010834298BF03F1FF30151DA0426B
:1010C00005DC01330220984205DB002038BD45F8DD
:1010D000041F0134F3E742F820100130F3E703283E
:1010E00013D1C80704D41320BDE8384000F030BA4B
:1010F0004910FF29F7D80432C3F30F1302EB83031F
:101100009A42E2D202F8011BFAE70B2000F020FA23
:10111000DBE700002DE9F8434E6816F001080F46A2
:1011200027D1042E25D9346804F00F03092B10D1E0
:101130007568C4F30F146D10AC4200D8651E396891
:10114000CB071AD54C10002C01DDA54220DA122065
:1011500034E0042B04D13046FFF7ACF90546EEE746
:10116000032B08D1C4F30F15C4F34174C4EB8505F8
:10117000E5E70025E3E74546E1E72F48FFF712FDE5
:10118000B0B109F055F890FBF5F404FB15040134F7
:10119000B8F1000F4ED1042E4CD9336803F00F0381
:1011A000092B11D1013456F824402046BDE8F883BC
:1011B00039682248FFF7F6FC20B91120BDE8F84352
:1011C00000F0C6B92C46E3E7042B2BD1304602F0E1
:1011D00015FA0546FFF798F9A042B8DB012C1BDC95
:1011E000304602F00BFA81462846FFF779F9461B94
:1011F000304602F019FC04460028D6D002F0FEF971
:101200008046786802F0FAF9A5EB090101443246FC
:10121000404608F0F9FCC8E72846FFF761F9013CB1
:101220000546DBE7032B05D13444E478640044F041
:101230000104BAE70B20C1E7F0B20000FBB20000E6
:101240002DE9F0414C6814F0010688462ED1042C9B
:101250002CD923688F6803F00F02092A13D165681F
:10126000C3F30F136D10AB4200D85D1ED8F8001009
:101270002848FFF797FC68B3236803F00F03092B96
:101280001ED1012317E0032A10D1FA0704D413203A
:10129000BDE8F04100F05CB97E10FF2EF7D8C3F333
:1012A0000F15C3F34173C3EB8505DFE70B20EFE7B1
:1012B000013344F823709D42FADA0020BDE8F08142
:1012C000032BFAD1033401239D42F6DB04F8016FAE
:1012D0000133F9E7D8F80010CB0706D549100029EB
:1012E00001DD8D4208DA1220D2E70B48FFF75AFCE5
:1012F00008B91120CCE72946236803F00F03092B16
:1013000003D1013144F82170D7E7032B04BF6418DF
:10131000E670D2E7F7B20000FBB20000086808B53B
:10132000C3071BD4042819D9036803F00F02092A44
:1013300001D1406808BD032A09D1C3F30F12C3F3DA
:101340004170C0EB8200400040F00100F2E7042A47
:1013500004D102F053F9FFF7D7F8F4E70B20BDE80A
:10136000084000F0F5B80000024A03480B2103F0E2
:1013700099BF00BF98B2000090B2000000207047F3
:101380000420704701207047002002F04DBB002070
:1013900070470020704700207047002070470020F1
:1013A0007047002070470020704700207047000001
:1013B000024A03480C2103F075BF00BF80B3000050
:1013C000E0B3000010B510F0010402D04410204634
:1013D00010BD042812D9026802F00F02042A07D1B6
:1013E00002F00CF90A222146BDE8104009F092B83B
:1013F000032A03D10A2221460430F5E7014B0D22CE
:101400001A70E4E77402002010F0010210B516D142
:10141000042802D90268C2F30F1211F0010310D19F
:10142000042902D90B68C3F30F13934216D1043079
:1014300000EB83020331904205D301200BE0002230
:10144000EBE70023F1E710F8014B11F8013F1CB95D
:10145000B3FA83F0400910BD9C42ECD00020FAE7BB
:101460002DE9F74F804689469A46304F304E6AB193
:1014700002233B70012333603368DFF8D0B00024CF
:10148000FC54444504DB03B0BDE8F08F3260F3E761
:1014900059F824003168C30707EB0105C1F548710D
:1014A00005D5244A4310284608F0F6FE04E0C8B9E2
:1014B000214A284608F0F0FE1C4808F067FF30601B
:1014C000BAF1000F0CD008F1FF33A34208DDB0F5EC
:1014D000487F05D2431C20223A540022FA5433603C
:1014E0000134CEE7042801D1144AE2E71BD902688F
:1014F00002F00F03042B06D1019102F07FF8104A8D
:1015000001990346CFE7092B03D143685A465B1084
:10151000C9E7032B08D1C2F30F13C2F34172C2EB28
:101520008303084ABFE70123074ABCE7750200208E
:101530009805002030BD000000B3000006B3000095
:101540005BC300005FB600006AB6000050B6000042
:10155000014B1870002070477402002010B501F094
:1015600091FD084C231D01461F22184608F028FF54
:1015700008F00CFF04308008000140F004002060F7
:10158000204610BD500200202DE9F04F85B000F13B
:10159000180104690291D0E90232824601EB840409
:1015A000BD4F4169029800EB8109397803EB820550
:1015B00029BB53F82230B94A1E1203F07F030435C9
:1015C00052F82330904643F0010318479AF801007F
:1015D00004F0AEFA00238AF8003021E03B7873B9BA
:1015E0002B681E1203F07F03043558F82330EAE716
:1015F000029B221DD31AD82B26DD1A233B70DAF862
:1016000008209AF8023039789AF80100AA1A921044
:1016100043EA022204F092FA00238AF800303B7079
:10162000DAF80830ED1A029BE41AA9EB0309AD10B1
:10163000A4104FEAA903CAF80C50CAF81040CAF81F
:10164000143005B0BDE8F08F3B7826600BB114462E
:10165000D5E72B681E1203F07F03144658F8233099
:101660000435B0E7029B221DD31AD82B02DD1A23C2
:101670003B70C4E72968216039782B1D11B11446ED
:101680001D46BCE76B681E1203F07F03144658F832
:101690002330083597E7029B221DD31AD82B02DD91
:1016A0001A233B70ABE73B7805EB860626600BB14F
:1016B0001446A4E72B681E1203F07F03144658F863
:1016C000233004357FE7029B221DD31AD82B02DD7D
:1016D0001A233B7093E7724B53F8263023603B7814
:1016E0000BB114468BE72B681E1203F07F031446E0
:1016F00058F82330043566E7694B54F8042D43F855
:1017000026203B78002B7FF47AAF2B681E1203F063
:101710007F03043558F8233055E7614B009353F8A5
:101720002600FFF74FFE834654F8040DFFF74AFEEC
:101730005844009B400040F0010043F826003B78ED
:10174000002B7FF45CAF2B681E1203F07F0304357F
:1017500058F8233037E7029B221DD31AD82B02DD1D
:101760001A233B704BE7029B4B4534BF59F80C3CA6
:10177000012323603B780BB1144640E72B681E120F
:1017800003F07F03144658F8233004351BE7029B0F
:10179000221DD31AD82B02DD1A233B702FE7029BA0
:1017A0004B450FD259F80C3C06F180465B10C3EB59
:1017B0008373033E334459F8233023603B782BB1C5
:1017C00014461CE718233B700023F6E72B681E1213
:1017D00003F07F03144658F823300435F3E6029BE8
:1017E0004B4519D259F80C3C54F8042C5B1006F107
:1017F0008046C3EB8373033E3344043C49F8232003
:101800003B78002B7FF4FBAE2B681E1203F07F03A6
:10181000043558F82330D6E618233B70F0E7029BD6
:101820004B452DD259F80C3C06F180465B10033E27
:10183000C3EB8373334459F82300FFF7C3FD221F22
:10184000834654F8040C0092FFF7BCFD59F80C3C99
:10185000009A5B10C3EB837358441E44400040F071
:10186000010049F8260014463B78002B7FF4C7AEF0
:101870002B681E1203F07F03043558F82330A2E6CC
:1018800018233B70F0E7029B221DD31AD82B09DDE9
:101890001A233B70B3E600BF7402002050B400006E
:1018A000C48B012059F8263023603B780BB11446D5
:1018B000A5E62B681E1203F07F03144658F8233068
:1018C000043580E654F8043D49F826303B78002B77
:1018D0007FF495AE2B681E1203F07F03043558F891
:1018E000233070E659F826004FEA600B54F8040DD7
:1018F000FFF768FD584440003B7840F0010049F88C
:101900002600002B7FF47BAE2B681E1203F07F03B2
:10191000043558F8233056E6029BA4EB8604A34214
:101920000BD83B78002B7FF46AAE2B681E1203F0B5
:101930007F03043558F8233045E6C34801F04EFED6
:101940003B78002B7FF45BAE2B681E1203F07F0305
:10195000043558F8233036E6002E05EB8605FFF6F1
:101960005FAE3B78002B7FF44AAE2B681E1203F06B
:101970007F03043558F8233025E654F8043D042B42
:1019800004D1002E05EB8605FFF64AAE3B78002B0E
:101990007FF435AE2B681E1203F07F03043558F830
:1019A000233010E654F8043D042B04D0002E05EB40
:1019B0008605FFF635AE3B78002B7FF420AE2B6812
:1019C0001E1203F07F03043558F82330FBE554F86A
:1019D000040CC3070BD54010013800280ADB400077
:1019E00040F0010005EB860544F8040C18E6FFF70B
:1019F000E9FCF1E73B78043C002B7FF400AE2B6858
:101A00001E1203F07F03043558F82330DBE5029BF8
:101A100004F10C02D31AD82B02DD1A233B70EEE539
:101A2000730003F4FF7343F001032360DAF8083016
:101A3000EB1A9D109AF8023043EA05235B0043F04D
:101A400001036360029BA9EB03035B1043F00103F6
:101A5000A3603412E6B27D4B8AF8024091463A7890
:101A600053F83630CAF808301AB103F108054C466D
:101A7000C5E503F10C059B681E1203F07F034C467D
:101A800058F823309FE5029B54F8046C4B452AD14B
:101A9000F1071BD4042E12D9336803F00F03042B73
:101AA0000ED1304601F0AAFD08F070FC063064301B
:101AB00003F034FC70B9043DDDF80890B0E507D0C0
:101AC000002E14BF4FF400700720F0E70A20EEE765
:101AD0000720ECE731469AF8010004F046F80023AD
:101AE0008AF80030E8E759F80C3C58495A106FF072
:101AF000030353430C3B09EB030449F8036059F813
:101B0000083C5A108AF80220D2B2C3F3552351F888
:101B10003220CAF8082059F8041C4FEA61090299DA
:101B200001EB89093978043402EB830500297FF43D
:101B300066AD52F823301E1203F07F03043558F8C7
:101B4000233040E554F8040CFFF73CFC1E28834684
:101B5000A4EB860425DC00280BDC3B78002B7FF40B
:101B60004EAD2B681E1203F07F03043558F8233066
:101B700029E501F077FAABF1030B354E834401F010
:101B800071FAA0EB0B00B042F9D83B78002B7FF440
:101B900036AD2B681E1203F07F03043558F823304E
:101BA00011E501238AF8003001F05CFA0A38584444
:101BB000CAF8040034E554F8040CFFF703FCA4EB66
:101BC0008604061E0BDC3B78002B7FF418AD2B68D7
:101BD0001E1203F07F03043558F82330F3E41D4B45
:101BE0009E4202DD1D233B7009E501238AF8003087
:101BF00001F038FA4FF47A7303FB06000A38D7E78E
:101C000000233046A4EB8604134E1A462146FFF704
:101C100027FC3168114801F00EFF114B3168186044
:101C20000E4803F04BFE31680C4803F0A3FF3B78ED
:101C3000002B7FF4E4AC2B681E1203F07F03043505
:101C400058F82330BFE400BF7CB60000CC830120ED
:101C50003F420F0080EE36009805002075020020FC
:101C6000080000203B78A4EB8604002B7FF4C7AC6F
:101C70002B681E1203F07F03043558F82330A2E4CA
:101C8000504603F0AFFB3B78002B7FF4B8AC2B68D9
:101C90001E1203F07F03043558F8233093E454F800
:101CA000043CB3BB54F80C3CDA0726D55B105A0051
:101CB00042F0010244F8082C002B3BDD5A0042F0B0
:101CC000010244F8042C54F8082CC3EB620354F8C6
:101CD0000C2CD10720D501335B0043F0010349F8F8
:101CE00026303B78002B7FF48AAC2B681E1203F061
:101CF0007F03043558F8233065E4042B06D91A68AD
:101D000002F00F02092A01D15B68CFE719233B706B
:101D100075E45B10013BCFE7042A08D9116801F094
:101D20000F01092903D1023352F82330D7E71923D1
:101D30003B7064E40435D4E7029A04EB86039B1AF3
:101D4000D82B10DC0122002E06F1FF330EDC3B788D
:101D5000002B7FF454AC2B681E1203F07F03043574
:101D600058F823302FE41A233B7048E422601E46C3
:101D70000434E8E7029A231D9B1AD82B02DD1A23AC
:101D80003B703CE4029B4B452AD254F8040CFFF70D
:101D900019FB002821DD59F80C3C5B1083421CDB49
:101DA000C3EB8373184400F180400438A4EB86032E
:101DB00059F820201A606FF0030303FB06443B78B8
:101DC0000434002B7FF41BAC2B681E1203F07F033E
:101DD000043558F82330FFF7F6BB20233B70EAE7C1
:101DE0001823FBE7C04B1A68A4EB86031A606FF058
:101DF000030303FB06443B780434002B7FF4FFAB62
:101E00002B681E1203F07F03043558F82330FFF7C8
:101E1000DABB54F8043C042B3B780CBF05EB860579
:101E2000043C002B7FF4EBAB2B681E1203F07F0306
:101E3000043558F82330FFF7C6BB54F8043C042B94
:101E40001CBF002344F8043C3B78A4F104021CBFEF
:101E500005EB8605224613B11446FFF7D0BB2B686D
:101E60001E1203F07F03144658F823300435FFF7A1
:101E7000AABB002EA4EB860115DC1C233B700022BC
:101E80006FF0030303FB06443B780A600434002B25
:101E90007FF4B5AB2B681E1203F07F03043558F8AE
:101EA0002330FFF790BB0B684FF0000C5B1051F82C
:101EB0002C0010F0010202D10D233B70E0E740102E
:101EC00083420CF1010CA8BF03466645EFDC5B00C2
:101ED00043F00102D4E7002EA4EB860115DC1C239D
:101EE0003B7000226FF0030303FB06443B780A605B
:101EF0000434002B7FF483AB2B681E1203F07F03A6
:101F0000043558F82330FFF75EBB0B684FF0000C28
:101F10005B1051F82C0010F0010202D10D233B7030
:101F2000E0E7401083420CF1010CB8BF0346664560
:101F3000EFDC5B0043F00102D4E754F8080CFFF734
:101F400041FA834654F8040CFFF73CFAA4EB8603ED
:101F50008345B4BF0420002018606FF0030303FB27
:101F600006443B780434002B7FF449AB2B681E12E7
:101F700003F07F03043558F82330FFF724BB54F8EF
:101F8000080CFFF71FFA834654F8040CFFF71AFAFF
:101F9000A4EB86038345D4BF0420002018606FF0B3
:101FA000030303FB06443B780434002B7FF427AB88
:101FB0002B681E1203F07F03043558F82330FFF717
:101FC00002BB54E902014FEA860B8142A4EB0B0BE2
:101FD00014D10423CBF800306FF0030303FB064455
:101FE0003B780434002B7FF40AAB2B681E1203F0FD
:101FF0007F03043558F82330FFF7E5BA042801D8E9
:102000000023E7E7C307FBD4036803F00F03042BA7
:10201000F6D1CB07F4D40429F2D90B6803F00F03EF
:10202000042BEDD1FFF7F0F900280CBF00230423A7
:10203000D0E754E902014FEA860B8142A4EB0B0B77
:1020400014D10023CBF800306FF0030303FB0644E8
:102050003B780434002B7FF4D2AA2B681E1203F0C5
:102060007F03043558F82330FFF7ADBA042801D8B0
:102070000423E7E7C307FBD4036803F00F03042B33
:10208000F6D1CB07F4D40429F2D90B6803F00F037F
:10209000042BEDD1FFF7B8F900280CBF042300236F
:1020A000D0E754F8080CFFF78DF9834654F8040C78
:1020B000FFF788F9A4EB86038345ACBF042000201A
:1020C00018606FF0030303FB06443B780434002BD5
:1020D0007FF495AA2B681E1203F07F03043558F88D
:1020E0002330FFF770BA00BF0800002054F8080C36
:1020F000FFF768F9834654F8040CFFF763F9A4EB83
:1021000086038345CCBF0420002018606FF00303D2
:1021100003FB06443B780434002B7FF470AA2B6841
:102120001E1203F07F03043558F82330FFF74BBA33
:1021300054F8043C042BA4EB860314BF04220022B1
:102140001A606FF0030303FB06443B780434002B52
:102150007FF455AA2B681E1203F07F03043558F84C
:102160002330FFF730BA54F8080CFFF72BF98346F9
:1021700054F8040CFFF726F95844A4EB86034000FA
:1021800040F0010018606FF0030303FB06443B7846
:102190000434002B7FF433AA2B681E1203F07F0354
:1021A000043558F82330FFF70EBA54F8080CFFF73F
:1021B00009F9834654F8040CFFF704F9ABEB00006F
:1021C000A4EB8603400040F0010018606FF00303A9
:1021D00003FB06443B780434002B7FF410AA2B68E1
:1021E0001E1203F07F03043558F82330FFF7EBB9D4
:1021F00054F8080CFFF7E6F8834654F8040CFFF790
:10220000E1F800FB0BF0A4EB8603400040F0010076
:1022100018606FF0030303FB06443B780434002B83
:102220007FF4EDA92B681E1203F07F03043558F8E4
:102230002330FFF7C8B954F8040CFFF7C3F88346FE
:10224000B8B91F233B70A4EB8603C3F800B06FF04E
:10225000030303FB06443B780434002B7FF4CFA92F
:102260002B681E1203F07F03043558F82330FFF764
:10227000AAB954F8080CFFF7A5F890FBFBFB4FEA4E
:102280004B0B4BF0010BDEE754F8040CFFF79AF808
:102290008346B8B91F233B70A4EB8603C3F800B094
:1022A0006FF0030303FB06443B780434002B7FF4F8
:1022B000A6A92B681E1203F07F03043558F82330BB
:1022C000FFF781B954F8080CFFF77CF890FBFBF39B
:1022D00003FB1B0B4FEA4B0B4BF0010BDCE754F8F5
:1022E000040CFFF76FF80028B8BF4042A4EB860348
:1022F000400040F0010018606FF0030303FB064448
:102300003B780434002B7FF47AA92B681E1203F06B
:102310007F03043558F82330FFF755B9A4EB860B3B
:10232000012EDBF8000028D1FFF74CF832460346B7
:102330000393009207F07CFF039B009A012BB8BF28
:10234000012390FBF3F101FB130313445B0043F003
:102350000103CBF800306FF0030303FB06443B7826
:102360000434002B7FF44BA92B681E1203F07F036B
:10237000043558F82330FFF726B9FFF723F800900B
:10238000DBF80400FFF71EF8009A0130831ACFE74C
:10239000A4EB860B5946304601F0E2FC6FF00303D4
:1023A00003FB06443B78CBF800000434002B7FF499
:1023B00026A92B681E1203F07F03043558F823303A
:1023C000FFF701B954F8080CFEF7FCFF834654F8F8
:1023D000040CFEF7F7FF0BEA0000A4EB86034000B5
:1023E00040F0010018606FF0030303FB06443B78E4
:1023F0000434002B7FF403A92B681E1203F07F0323
:10240000043558F82330FFF7DEB854F8080CFEF70F
:10241000D9FF834654F8040CFEF7D4FF4BEA0000C2
:10242000A4EB8603400040F0010018606FF0030346
:1024300003FB06443B780434002B7FF4E0A82B68B0
:102440001E1203F07F03043558F82330FFF7BBB8A2
:1024500054F8080CFEF7B6FF834654F8040CFEF758
:10246000B1FF8BEA0000A4EB8603400040F00100BE
:1024700018606FF0030303FB06443B780434002B21
:102480007FF4BDA82B681E1203F07F03043558F8B3
:102490002330FFF798B854F8040CFEF793FFC043BD
:1024A000A4EB8603400040F0010018606FF00303C6
:1024B00003FB06443B780434002B7FF4A0A82B6870
:1024C0001E1203F07F03043558F82330FFF77BB862
:1024D00054F8080CFEF776FF834654F8040CFEF718
:1024E00071FF0BFA00F0A4EB8603400040F00100FE
:1024F00018606FF0030303FB06443B780434002BA1
:102500007FF47DA82B681E1203F07F03043558F872
:102510002330FFF758B854F8080CFEF753FF8346F2
:1025200054F8040CFEF74EFF4BFA00F0A4EB8603C0
:10253000400040F0010018606FF0030303FB064405
:102540003B780434002B7FF45AA82B681E1203F04A
:102550007F03043558F82330FFF735B854F80C0CD6
:10256000FEF730FF834654F8080CFEF72BFF8BFB79
:10257000002354F8040CCDE90023FEF723FFDDE926
:102580000023C0F1200CB0F1200103FA0CFC22FA68
:1025900000F040EA0C005CBF43FA01F108436FF021
:1025A0000303A4EB860E400003FB06443B7840F097
:1025B0000100CEF800000434002B7FF420A82B6823
:1025C0001E1203F07F03043558F82330FEF7FBBFDB
:1025D000A4EB860B59463046FEF744FD6FF003032B
:1025E00003FB06443B78CBF800000434002B7FF457
:1025F00006A82B681E1203F07F03043558F8233019
:10260000FEF7E1BFA4EB860421463046FEF741FD0C
:102610003B78002B7EF4F3AF2B681E1203F07F0390
:10262000043558F82330FEF7CEBFA4EB860B59468D
:102630003046FEF76FFD6FF0030303FB06443B7863
:10264000CBF800000434002B7EF4D9AF2B681E12A7
:1026500003F07F03043558F82330FEF7B4BFA4EB32
:10266000860421463046FEF7EBFD3B78002B7EF4D6
:10267000C6AF2B681E1203F07F03043558F82330D1
:10268000FEF7A1BFA4EB860B59463046FEF746FE87
:102690006FF0030303FB06443B78CBF800000434DF
:1026A000002B7EF4ACAF2B681E1203F07F030435C1
:1026B00058F82330FEF787BF54F8040C00F09EFF53
:1026C00054F8083CDA072AD4042B0CD91B6803F011
:1026D0000F03013B082B10D8DFE803F00521272367
:1026E0000F0F0F0F2500C74907F046FEA4EB860326
:1026F000002814BF002204221A606FF0030303FBBA
:1027000006443B780434002B7EF479AF2B681E120C
:1027100003F07F03043558F82330FEF754BFBA495D
:10272000E2E7BA49E0E7BA49DEE7BA49DCE7029BEB
:1027300004F1040BABEB0303D82B03DD1A233B702E
:10274000FEF75DBF00F096FC3B78400040F00100D2
:10275000206013B15C46FEF752BF2B681E1203F0D7
:102760007F035C4658F823300435FEF72CBF029BEC
:1027700004F1040BABEB0303D82B03DD1A233B70EE
:10278000FEF73DBF00F06EFCA34B03EA40003B7830
:1027900040F00100206013B15C46FEF730BF2B68AB
:1027A0001E1203F07F035C4658F823300435FEF711
:1027B0000ABF029B04F1040BABEB0303D82B03DD30
:1027C0001A233B70FEF71BBF00F054FC934B1B68B1
:1027D00098423DBFC3F5830303F63713C018C01AF0
:1027E00040003B7840F00100206013B15C46FEF7EA
:1027F00006BF2B681E1203F07F035C4658F8233097
:102800000435FEF7E0BE00F035FC844B18603B78E1
:10281000A4EB8604002B7EF4F2AE2B681E1203F0AC
:102820007F03043558F82330FEF7CDBE3046A4EBC5
:10283000860701237A4E1A463946FEF711FE3068A4
:10284000643002F06BFD10B9043DFEF7E9BE9AF862
:1028500001203168734803F09CF901238AF80030A5
:1028600000F000FC704A33681268063302FB030074
:10287000CAF804003C46FEF7D3BE3046A4EB8607F8
:10288000674E012300223946FEF7EAFD30686430C6
:1028900002F044FD0028D7D0624802F0FBFEDCE7DE
:1028A000FEF75CFE6FF00303A4EB860B03FB06440C
:1028B0003B78CBF800000434002B7EF4A0AE2B68EC
:1028C0001E1203F07F03043558F82330FEF77BBE59
:1028D0003B78A4EB8604002B7EF491AE2B681E128D
:1028E00003F07F03043558F82330FEF76CBEA4EBE9
:1028F000860B584600F0EDFB6FF0030303FB064424
:102900003B78CBF800000434002B7EF478AE2B68C3
:102910001E1203F07F03043558F82330FEF753BE30
:10292000A4EB860B584600F0D6FB6FF0030303FBC5
:1029300006443B78CBF800000434002B7EF45FAEF5
:102940002B681E1203F07F03043558F82330FEF77E
:102950003ABEA4EB860B5946304600F0BFFB6FF041
:10296000030303FB06443B78CBF800000434002B40
:102970007EF445AE2B681E1203F07F03043558F831
:102980002330FEF720BEA4EB8604204600F0D8FBDF
:102990003B78002B7EF433AE2B681E1203F07F03CE
:1029A000043558F82330FEF70EBEA4EB860B5946CB
:1029B000304600F0FFFB6FF0030303FB06443B7857
:1029C000CBF800000434002B7EF419AE2B681E12E5
:1029D00003F07F03043558F82330FEF7F4BDA4EB71
:1029E0008604204600F04CFC3B78002B7EF407AEBA
:1029F0002B681E1203F07F03043558F82330FEF7CE
:102A0000E2BD00BF8CB6000094B600009BB600008B
:102A1000A2B60000A7B60000FEFFFF7FA0050020C1
:102A20009805002075020020040000200121304696
:102A300000F0EAFB3B78002B7EF4E1AD2B681E1220
:102A400003F07F03043558F82330FEF7BCBD0021A6
:102A5000304600F0D9FB3B78002B7EF4D0AD2B68DC
:102A60001E1203F07F03043558F82330FEF7ABBD88
:102A7000A4EB860B584600F029FC6FF0030303FB20
:102A800006443B78CBF800000434002B7EF4B7AD4D
:102A90002B681E1203F07F03043558F82330FEF72D
:102AA00092BDA4EB860B584600F024FC6FF00303A4
:102AB00003FB06443B78CBF800000434002B7EF483
:102AC0009EAD2B681E1203F07F03043558F82330A7
:102AD000FEF779BDA4EB8604204600F0DFFB3B78CF
:102AE000002B7EF48CAD2B681E1203F07F0304359F
:102AF00058F82330FEF767BDA4EB8604204603F0A8
:102B0000F1FB3B78002B7EF47AAD2B681E1203F0AC
:102B10007F03043558F82330FEF755BDA4EB860B30
:102B2000584603F075FC6FF0030303FB06443B7843
:102B3000CBF800000434002B7EF461AD2B681E122C
:102B400003F07F03043558F82330FEF73CBDA4EBB7
:102B50008604204603F03CFB3B78002B7EF44FAD0F
:102B60002B681E1203F07F03043558F82330FEF75C
:102B70002ABDA4EB860B584603F042FB6FF003031B
:102B800003FB06443B78CBF800000434002B7EF4B2
:102B900036AD2B681E1203F07F03043558F823303E
:102BA000FEF711BDA4EB86042146304601F06AFB16
:102BB0003B78002B7EF423AD2B681E1203F07F03BD
:102BC000043558F82330FEF7FEBCA4EB86042146FA
:102BD000304601F07DF93B78002B7EF410AD2B6878
:102BE0001E1203F07F03043558F82330FEF7EBBCC8
:102BF000A4EB86042146304601F07AFA3B78002B9C
:102C00007EF4FDAC2B681E1203F07F03043558F8E8
:102C10002330FEF7D8BCA4EB86042146304601F0F1
:102C20008DFA3B78002B7EF4EAAC2B681E1203F081
:102C30007F03043558F82330FEF7C5BCA4EB860BA0
:102C40005946304603F0BEFC6FF0030303FB064415
:102C50003B78CBF800000434002B7EF4D0AC2B681A
:102C60001E1203F07F03043558F82330FEF7ABBC87
:102C7000A4EB860B5946304603F0ACFC6FF003031F
:102C800003FB06443B78CBF800000434002B7EF4B1
:102C9000B6AC2B681E1203F07F03043558F82330BE
:102CA000FEF791BCA4EB860B5946304603F09AFC24
:102CB0006FF0030303FB06443B78CBF800000434B9
:102CC000002B7EF49CAC2B681E1203F07F030435AE
:102CD00058F82330FEF777BCA4EB860B59463046F4
:102CE00003F0C6F96FF0030303FB06443B78CBF80F
:102CF00000000434002B7EF482AC2B681E1203F01B
:102D00007F03043558F82330FEF75DBCA4EB86043E
:102D10002146304601F006F93B78002B7EF46FAC7B
:102D20002B681E1203F07F03043558F82330FEF79A
:102D30004ABCA4EB86042146304601F027FA3B78D2
:102D4000002B7EF45CAC2B681E1203F07F0304356D
:102D500058F82330FEF737BCA4EB860B59463046B3
:102D600001F08EF96FF0030303FB06443B78CBF8C8
:102D700000000434002B7EF442AC2B681E1203F0DA
:102D80007F03043558F82330FEF71DBCA4EB8604FE
:102D90002146304601F038F93B78002B7EF42FAC09
:102DA0002B681E1203F07F03043558F82330FEF71A
:102DB0000ABC029BE31A9B10A4EB8604CAF81030ED
:102DC0002146304602F0A6FC3B78002B7EF417AC7F
:102DD0002B681E1203F07F03043558F82330FEF7EA
:102DE000F2BB029BE31A9B10A4EB860BCAF81030CF
:102DF0005946304602F08EFC6FF0030303FB064495
:102E00003B78CBF800000434002B7EF4F8AB2B6841
:102E10001E1203F07F03043558F82330FEF7D3BBAE
:102E20002DE9F84F224D0023002B03F1FF3706DA7E
:102E300001F0CAFA02F098FD02F00AFF19270026F5
:102E4000DFF878803046D8F80020B24215DD2B68D4
:102E5000184C01339342A8BF00232B60D5F8009093
:102E6000F02303FB09F304EB030AE35CA346EBB195
:102E7000022B04D15046FEF787FB3B46D4E7012BDB
:102E80000ED108B900F0EEF8F02303FB09F39B44E0
:102E90000949DBF80420821A8A429CBF0222E254CC
:102EA000F02303FB09F3E35C022BE3D00136CAE70E
:102EB000000000206C7A01203F420F009C0500209A
:102EC0000B4B012200211A61C3F80415C3F8081541
:102ED0000421C3F810154FF44031C3F804131A60ED
:102EE000044B4FF480611960034B1A70704700BFA8
:102EF00000A0004000E100E0C7050020042070476A
:102F0000F8B5D1E9004514F001002DD015F001000D
:102F10002AD064101C2C3CD81F4F6D1041F288360B
:102F20003B5DAE42A8BF2E46012B05D001212046B5
:102F300004F086FD01233B55184B1B780BB9FFF7B6
:102F4000BFFF002D4FF00003154A0EDC154940F27B
:102F5000DC50FF25D65CB44204BF21F81300D554E1
:102F60000133042BF6D10420F8BDD15C8C4203D18F
:102F70000C4A22F81360F6E70133042BF5D1002345
:102F8000D15CFF2901D1D454F2E70133042BF7D1EE
:102F9000E9E70020E8E700BFA8050020C7050020FA
:102FA0001C0000200E00002070B5D1E9004514F08F
:102FB00001001BD015F0010018D064101D2C28BF93
:102FC0001B24164E335D012B05D00121204604F051
:102FD00037FD01233355124B6D10A5F110029A42B3
:102FE000104B04D94FF0FF321A60042070BD0E4A16
:102FF0001C600E4B93FBF5F313800D4A127812B947
:10300000FFF75EFFF1E70B4A01219164D2F8481502
:103010000B449BB2C2F84035E7E700BFA80500208B
:1030200090860100180000200C00002020A107005D
:10303000C705002000A00040002802DC1C20FEF78D
:1030400087BA0120704704207047002802DC1C204A
:10305000FEF77EBA0B68DB0701D40D20F8E70020ED
:1030600070470000024B01221A64D3F840057047F4
:103070000080004008B5FFF7F5FF4FF47A73B0FB0E
:10308000F3F008BD0048704708B700001D207047E6
:1030900070B5054D2B5C8B4204460E4602D004F001
:1030A000CFFC2E5570BD00BFA805002070B50024D0
:1030B000064D2646635D012B04D10021204604F015
:1030C000BFFC665501341D2CF4D170BDA80500204D
:1030D00070470F2070473B2070470000F8B50B6821
:1030E000DA0707460D4604D40D20FEF731FA012019
:1030F00007E05B10062B05D103F090F8400040F08C
:103100000100F8BDF3D80C4A0C4E52F82340335D51
:103110002BB10021204604F093FC00233355012FEE
:1031200006DD6B68042B03D10221204604F088FCE5
:10313000204604F08FFBE1E7ECB60000A805002074
:1031400070B50468E20702D54568EB0704D40D208A
:10315000BDE87040FEF7FCB964101C2C23D8124E59
:10316000335D012B18D00121204604F069FC0123B6
:103170001B2C335510D10D4BDA6E0D4B202AB8BFE6
:103180004FF0A04302F01F0203EB8203D3F80027A5
:1031900042F44072C3F80027A5F34A012046BDE877
:1031A000704004F0FBBB70BDA80500207CC6000089
:1031B0000003005070B50C68E30704D40D20FEF73F
:1031C000C7F9012070BD64101C2C14D8012814DD2F
:1031D0004B68042B14BF002502250A4E335DAB4219
:1031E00004D02946204604F02BFC3555204604F037
:1031F0006DFC012803D00020E4E70025EDE7042062
:10320000E0E700BFA80500201C2870B504460D4665
:103210002CD8174E335C012B04D0012104F010FC94
:10322000012333551C2C19D1124A0123536002F596
:10323000A042536002F5805253600F4B1A6F0F4B40
:10324000202AB8BF4FF0A04302F01F0203EB820315
:10325000D3F8002742F44072C3F80027291C204607
:1032600018BF0121BDE8704004F014BC70BD00BF60
:10327000A805002000C001407CC6000000030050EB
:103280000368D90702D40D20FEF762B941680A1F0E
:10329000514251415810FFF7B7BF000013B50A4A19
:1032A000044692E8030022686B46042A83E8030080
:1032B00019464FF0020003D100F01AFF02B010BD12
:1032C00000F03CFFFAE700BFB4B6000010B5084CB0
:1032D00063792BB10021052004F0B2FB0023637158
:1032E000052004F0F3FB00280CBF0420002010BDD3
:1032F000A805002010B5084CE37A2BB100210B2063
:1033000004F09EFB0023E3720B2004F0DFFB002897
:103310000CBF0420002010BDA8050020F8B5314CDA
:10332000D4F84031B3B10023D4F84055C4F840314B
:103330002D4B186800280DDB2C4A1178B1FA81F169
:103340004909117004F0A6FB294B1B882B449BB242
:10335000C4F84035234AD2F84431002B37D000213D
:10336000244ED2F84445C2F844113378224D0C342F
:1033700033B12B68032B03D8204AD05C04F08AFBBE
:103380002B681E4F01335A4202F0030203F003037D
:1033900058BF53422B600022042B194618D001332A
:1033A000F81810F8010CFF2801D10122F4E702B14E
:1033B0002960012104F06EFB012333702A68104B51
:1033C00033F812302344074A9BB2C2F84435F8BDA3
:1033D0004FF0FF332B600023337004F58C435033E0
:1033E000F1E700BF00A0004018000020C605002043
:1033F0000C000020C5050020A40500201C000020B2
:103400000E000020094B0A4940F2DC521A805A8013
:103410009A80DA80074A00231370074AFF20087059
:1034200048708870C8701360704700BF0E0000209D
:103430001C000020C5050020A4050020024B4FF011
:10344000FF321A60704700BF18000020024A03488C
:10345000062101F027BF00BFBCB6000062BE00001D
:1034600038B54FF4E1311D4803F0D2FF1C4B032166
:103470000122C3F80815002404211A61C3F81015AD
:103480001A60C3F804454FF080430221C3F81815B1
:103490000A209A6004F0D8F9124A2346FF21995471
:1034A00001331D2BFBD1104B104D01221A6000205F
:1034B0000F4A042301461468002CFCD02C681160CC
:1034C000013B44EA0020F6D10A4B01221A6004F0C5
:1034D000F9F8BDE8384000F0F9BF00BFEC790120F1
:1034E00000800040A805002000D0004008D5004022
:1034F00000D1004004D00040F8B506460948094F05
:103500000C4603F0C5FF8442A8BF04463546AB1BFA
:103510009C4205DD384603F0C1FF05F8010BF6E7D4
:103520002046F8BDEC7901200146014803F075BF43
:10353000EC790120C3070CD4064B1B68834208D8E2
:10354000054B1B68984204D850F8043C002B18BF68
:1035500018467047D0050020CC0500200B4908B55F
:103560000122002341F823200133642BFAD1084BB8
:103570001A60084B084A1846002106F069FB074B01
:1035800040F8043F064B186008BD00BFC48B012003
:1035900008000020D405002070670100A09D0500F0
:1035A000C8050020034B044A1A60044B044A1A6001
:1035B000FFF7D4BFD0050020D4050020CC050020A3
:1035C000446D0120044B1B681868C0F30F100238CB
:1035D00020EAE070704700BFC805002000B59BB02E
:1035E0000246054901A806F08BFE01A802F06FF81B
:1035F00002F02EFBFCE700BF8FB70000C30713D417
:10360000042802D812D00B487047036803F00F0358
:10361000042B01D104307047092B09D0064A074812
:10362000032B18BF10467047054870470548704780
:103630000548704700B300007AB7000083B7000068
:1036400069B7000006B3000073B70000064B0749D6
:1036500000201A6843F8040CC2F30F12023203EB85
:1036600082038B42F5D37047D8050020446D0120BA
:103670002F4B304A1868304B2DE9F0411C682F4D14
:10368000136803F00F01072928D81368C3F30F1339
:10369000023302EB8302AA42F2D32949002251F8F5
:1036A0002200FFF747FF41F822000132642AF6D1D9
:1036B000244A1068FFF73EFF1060234A106810B1DB
:1036C000FFF738FF1060214B214C1E680021F027C6
:1036D0004FF03C08B14214DBBDE8F081C3F30F1397
:1036E00002EB83039A42D0D01968CE0707D48842F0
:1036F00005D28C4203D351F8041C01B11960043B7C
:10370000F0E707FB01F31A191B5D0BB90131E1E783
:103710001269551E08FB012204EB82021832002DAB
:10372000F4DB52F8040DFFF705FF013D1060F6E7EA
:10373000D0050020D8050020CC050020446D0120D4
:10374000C48B012008000020446D01209C0500204E
:103750006C7A0120C307F0B540D4214B1C68A0420D
:103760003CD3204B1D68A84238D850F8043CABBB72
:1037700003680246C3F30F13012673B9904242F85F
:10378000046C2BD0116851F8043C51F82370176079
:1037900041F82320013B0A46EFE752F82310CF07F8
:1037A00002EB830C18D48C4216D88D4214D351F8F6
:1037B000047C8FB90F6807F00F0EBEF1070F08D910
:1037C000CCF8007042F8043C0B680A60C3F30F1396
:1037D000E1E741F8046CD0E7013BCEE7F0BD00BF64
:1037E000D0050020CC0500200D4930B50D4C0B460E
:1037F0001A6853F8045CC2F30F12901C65B18B4237
:1038000014BF0A46002243F8042C01EB800103EBAD
:103810008003A342ECD330BD12011A60F7E700BF6A
:10382000D8050020446D0120144B2DE9F041144CC3
:103830001E464FF000083268C2F30F1712070FD070
:103840007D1C9E424FEA850505D018462A46314622
:1038500006F0E5F903465A1904352B44C2F80080F6
:10386000023706EB8706A642E5D3E41AA410013C12
:10387000044A24011C601360BDE8F081D8050020D3
:10388000446D0120C80500202DE9F0419AB0FFF7F2
:10389000E9FB214D0746002455F824000134FFF7C9
:1038A00059FF642CF8D11D4B1868FFF753FF1C4BD0
:1038B000186808B1FFF74EFF1A4DDFF87480002634
:1038C000D8F800309E4218DBFFF78EFFFFF7D0FEDE
:1038D000FFF7AAFFFFF7C6FB134B14491B681B68D1
:1038E000C3F30F13C21B023B01A806F009FD01A898
:1038F00001F0EDFE1AB0BDE8F0812B7813B9013666
:10390000F035DDE72C69013C002CF8DB05EB840386
:103910009869FFF71FFFF6E7C48B0120080000201D
:10392000446D01206C7A0120C805002049B70000D1
:103930009C0500202DE9F8431B4C23681B684D1C97
:10394000C3F30F139D42064688461746A1460CDB7B
:10395000FFF79AFF23681B68C3F30F139D4204DB34
:103960000A20BDE8F843FDF7F3BD08F10202D9F8DB
:1039700000009B1A1B0140F82230002340F8043C51
:1039800006F00F06034646EA0816940043F8046B57
:103990000119083CC9F800101C44A34201D3BDE83A
:1039A000F88343F8047BF8E7C8050020F8B510F069
:1039B000010704460E462CD1174B1B68834228D8BA
:1039C000164B1B68834224D9154D286000680122DC
:1039D00000F00F00FFF7AEFF2C682F600546C0B166
:1039E0002146043051F8042BC2F30F12B242A8BF93
:1039F0003246920006F008F9FFF728FE44F8045C0E
:103A0000FFF736FE2268074B44F8047C134023601E
:103A10002C462046F8BD00BFD0050020CC05002074
:103A2000446D0120F0FF0F00011D0022042091FBD6
:103A3000F0F1FFF77FBF38B5054608460C46FFF7A3
:103A4000F3FF50B1C21C2B46591B8C4206DC002CE4
:103A5000ACBF0419041C0023237138BD13F8011BEB
:103A600002F8011FF0E7F0B502289BB00C4604DC19
:103A70001C20FDF76DFD1BB0F0BD0868C20706D421
:103A8000042804D9036803F00F03042B01D00E208F
:103A9000EFE74B6813F00107F9D1042BF7D91B6846
:103AA00003F00F03042BF2D18B68DB0701D40D2048
:103AB000DFE7FFF7A3FD06466068FFF79FFDA568F7
:103AC0001AAC014604F8647D6D10304602F04CFFDC
:103AD00029466423224602F0A9FF204606F056FC40
:103AE00001462046FFF7A7FFC5E7000010B50446D2
:103AF000ADF5806D10B9FFF797FF0BE002F05BFEAC
:103B00000138062827D8DFE800F008081017280435
:103B1000230000200DF5806D10BD204602F0C5FE8B
:103B2000011B2046FFF787FFF4E7204602F071FEF5
:103B3000400040F00100EDE769464FF48062204606
:103B400002F081FE684606F021FC01466846E9E77E
:103B500004210348E6E70020CDE70420DAE700BFB0
:103B6000D8B70000022838B50C4604DC1C20BDE89C
:103B70003840FDF7EDBC0868C10706D4042804D915
:103B8000036803F00F03042B01D00E20EFE76368F6
:103B9000DA07FAD4042BF8D91B6803F00F03042BBF
:103BA000F3D1A368DB0701D40D20E0E7FFF726FD82
:103BB00005466068FFF722FDA468014664102846A8
:103BC00002F0D2FE214602F00EFFBDE83840FFF7BA
:103BD0008DBF012838B50C4604DC1C20BDE83840F8
:103BE000FDF7B6BC0868C10706D4042804D90368E9
:103BF00003F00F03042B01D00E20EFE76368DA0710
:103C0000FAD4042BF8D91B6803F00F03042BF3D16B
:103C1000FFF7F4FC05466068FFF7F0FC0146284614
:103C200002F0A2FE02F01EFF400040F0010038BD8D
:103C3000012870B505460C4604DC1C20BDE8704028
:103C4000FDF786BC0868C10706D4042804D90368B8
:103C500003F00F03042B01D00E20EFE76368DA07AF
:103C6000FAD4042BF8D91B6803F00F03042BF3D10B
:103C7000FFF7C4FC06466068FFF7C0FC022D014652
:103C800015D0A468E30712D56410304602F06CFE2C
:103C9000054602F090FD012812D1002C02DD01350D
:103CA000012C07D12846BDE87040FFF71FBF4FF039
:103CB000FF34EAE7284602F006FE013C0546EFE73E
:103CC0000228EFD1002CEDDD0135012CEAD00022D5
:103CD0001146284602F021FE02F0F5FD013C0546A2
:103CE000F3E70000086810B510F001041AD0441082
:103CF00007EE904A9FED187AF8EEE77A67EE877A3A
:103D000017EE900A05F0E2FB03F0EAFF0022134BE6
:103D100005F034FC03F096FF05F0E0FE400040F0B3
:103D2000010010BD042812D9036803F00F03042B0F
:103D300007D1FFF763FC0A22214606F0EBFB04469D
:103D4000D6E7032B03D10A2221460430F5E70D20E4
:103D5000FDF7FEFBCCE700BFD30237390000D040AF
:103D6000086808B5C30706D4042804D9036803F01B
:103D70000F03042B04D00E20BDE80840FDF7E8BB7C
:103D8000FFF73CFC0378232B08BF013010220021F1
:103D900006F0C0FB00F10053B3F1804F01D31420B3
:103DA000EAE7400040F0010008BD0000024A034875
:103DB000062101F077BA00BFA8B70000A0B7000045
:103DC000002070471E20FDF7C3BB1E20FDF7C0BBBF
:103DD0001E20FDF7BDBB1E20FDF7BABB1E20FDF760
:103DE000B7BB1E20FDF7B4BB1E20FDF7B1BB1E20E4
:103DF000FDF7AEBB1E20FDF7ABBB1E20FDF7A8BB39
:103E0000024A03480B2101F04DBA00BF14B800006C
:103E10006CB80000034B01221A60034B18689040F5
:103E200010437047646D0120486D01202DE9F04179
:103E3000EFF31082012302F0010883F31088154983
:103E4000154C0968154D164E01398B4003274FF06C
:103E50000E0C4FF00B0E002B18D021682960184271
:103E60000AD0724611000139FDDC21683160390049
:103E70000139FDDC5B08EEE739000139FDDC216822
:103E80003160624611000139FDDCF3E788F31088E8
:103E9000BDE8F08120000020586D01200805005089
:103EA0000C05005070B5084E084D002456F824004B
:103EB0000021FFF7EDF855F8240000210134FFF749
:103EC000E7F8052CF2D170BD04B9000050BC000029
:103ED00008B5054B00221A60044B1B680BB102F0B9
:103EE00009FC002008BD00BF606D01205078012052
:103EF00010B5041E0ADA0024074B53F824200123CE
:103F00009340064A1360064A136010BDFFF7BEF8DF
:103F1000A042F0DDF0E700BF7CC60000586D012034
:103F2000180500502DE9F843344B1B680C461BB9AB
:103F30004FF0FF30FFF7DCFF246814F0010525D0B7
:103F4000C4F34743C4F34720C4F3470240F2596522
:103F500040435B4390FBF5F193FBF5F0000240EA30
:103F600001401346534393FBF5F31843244B1B685E
:103F7000202B01BF234BC4F3456453F8243043EA9C
:103F80000020FFF753FF0020BDE8F883042CFAD986
:103F9000236803F00F03092BF5D154F8046FDFF801
:103FA0006080DFF86090761040F25967B542EADA37
:103FB00054F8042FD3071FD5C2F34743C2F3472059
:103FC000C2F3470140435B4390FBF7FC93FBF7F0E0
:103FD000000240EA0C400B464B4393FBF7F31843B7
:103FE000D8F80030202B02BFC2F3456259F82230C6
:103FF00043EA0020FFF71AFF0135D7E7586D01208B
:1040000020000020F4BA000008B50B68DA074CBFA6
:104010005B104FF0FF3301280DDD4A68042A14BFFE
:1040200018222022054918460A60FFF751F8FFF7C9
:104030005FFF002008BD1822F4E700BF2000002029
:1040400010B510F0010402D04410204610BD042821
:1040500012D9026802F00F02042A07D1FFF7CEFA44
:104060000A222146BDE8104006F054BA032A03D1C3
:104070000A2221460430F5E70D20FDF769FAE4E74E
:10408000086810F0010370B51CD0FFF7D9FF034694
:10409000203B5E2B27D8154C03EB83030022012124
:1040A00010462344052A1AD09E5C052410252E4272
:1040B00018BF4018013C4FEA41014FEA6505F6D1AF
:1040C0000132EFE70428E3D9026802F00F01042966
:1040D000DED1C2F30F13002BDAD00379D8E740000A
:1040E00040F0010070BD0120FCE700BF18B90000DE
:1040F00038B508680D46FFF7A3FF04466868FFF768
:104100009FFF621E042A014612D8431E042B0FD8BB
:10411000084803EB830313440568012202FA03F302
:104120002B430360044B1B6813B1204602F0E3FAF3
:10413000002038BD606D01205078012038B5086836
:104140000D46FFF77DFF04466868FFF779FF621EA2
:10415000042A014614D8431E042B11D8094803EB46
:1041600083031344012202FA03F3026822EA0302E2
:10417000054B02601B681BB10022204602F0BBFA0F
:10418000002038BD606D0120507801202DE9F04FEE
:10419000054685B008680C46FFF752FF022D0190D6
:1041A0003CDD6068FFF74CFF0746A068FFF748FF5B
:1041B0000446231DDFF8C8A00293661E4FF00108D5
:1041C000029B9E4206F1010935D006EB8602531E82
:1041D00007F1050B3D460393AB4522D0042E19D8B9
:1041E0006A1E042A16D8039B019ADAF800005919AE
:1041F000224B4FF0010C18EA020E0CFA01F11B6879
:1042000011D00143CAF8001023B16246494628463E
:1042100002F071FA4FEA48080135DDE7012427462C
:10422000C7E74E46CCE720EA0101CAF80010002B90
:10423000F0D07246EAE73D1D042D1BD8012C19D1A0
:10424000DFF83C80DFF834900026D8F8003004FA1C
:1042500005F223EA0203C8F80030D9F8003001362D
:1042600023B100223146781D02F045FA052E05F1F2
:104270000505EAD1002005B0BDE8F08F5078012097
:10428000606D0120086808B5C30703D5FFF7D8FEA5
:10429000054B1860054B1B681BB1034B186802F0F7
:1042A0002BFA002008BD00BF606D0120507801206E
:1042B0002DE9F3413F4D4FF441732C68ADF80430C4
:1042C0000A238DF806305CBBFFF7ECFDDFF8F480C5
:1042D000264658F8267001213846FEF7D9FE0136E9
:1042E0000021384603F0D6FB052EF2D100260DF151
:1042F000040816F8087001213846FEF7C9FE013699
:104300000121384603F0C6FB032EF2D1FEF7AAFEC8
:10431000294B186001232B60204602B0BDE8F081D4
:10432000012C1CD1244C2668FEF79CFE864298BFC7
:10433000801BC72801D80024EEE700210420FEF7E7
:10434000A7FE00210320FEF7A3FE00210A20FEF7AE
:104350009FFEFEF787FE022320602B60EBE7022C16
:1043600021D1154B1C68FEF77DFE844298BF001BCF
:10437000B0F57A6FDFD3042003F06CFA0446032013
:1043800003F068FA06460A2003F064FA3444204435
:10439000C0F53F6003230D3090FBF3F0074B18602E
:1043A000012003F057FA064A00232B601360012412
:1043B000B2E700BF546D01205C6D0120486D012003
:1043C000646D012050BC00002DE9F843384E32687E
:1043D00052B9384B1B683BB9374B1B68002B5DD07B
:1043E000BDE8F843FFF764BF344D2C68CCB9324BBD
:1043F0001B68002B4ED12F4A3368106811460028E5
:104400004ED12F4F2F4E0B6057F824000021FEF79E
:104410003FFE56F8240001210134FEF739FE052C39
:10442000F2D12B68264EDFF88C90264F002BCCBFA4
:1044300003F1FF330423002156F82300FEF728FE82
:104440002A68214B53F82280002404EB840101EBFD
:104450000803D9F8001057F82400194101F00101B0
:10446000013403F017FB052CEFD12B68012156F81E
:104470002300FEF70DFE2B68002156F8230003F001
:1044800009FB2B68013393FBF4F404EB84041C1B3D
:104490002C6003E0FFF70CFF0028ACD1BDE8F883E7
:1044A000002BAED11360BDE8F843FFF7FBBC00BFA3
:1044B000606D0120506D0120646D01204C6D012064
:1044C00004B9000050BC0000F4BB00004FF0FF3006
:1044D000FFF70EBD024A0348092100F0E3BE00BF0A
:1044E00008BC000064BC00004FF0805310B51A698E
:1044F000094B0224C3F8044522F00302884203D387
:104500000022C3F8042510BDD3F80044002CFBD0D2
:10451000C3F808051044F1E700E00140002815BF8A
:104520004FF4D2214FF4B4214FF4B4204FF496202D
:10453000FFF7DABF00280CBF4FF496234FF4B423E3
:104540001868030E532B0CBF20F07F4000207047EB
:10455000064B0122C3F80425D3F80024002AFBD01F
:1045600000220160C3F80425704700BF00E001404D
:10457000002821F07F4141F0A6410CBF4FF4962066
:104580004FF4B420FFF7E4BF0A4B30B50124C3F861
:104590000445002903DC0022C3F8042530BD52F88D
:1045A000044BD3F80054002DFBD040F8044B0139E4
:1045B000EFE700BF00E0014038B54C680234054623
:1045C0000A462146FFF7E0FF05EB840038BD0000F6
:1045D000124B1B68002B0BBF4FF4B4224FF4D222B6
:1045E0004FF496234FF4B42328B91A1DDB79522BCC
:1045F00008BF1046704782420DD9C378522B0AD1AA
:104600004368023300EB8300824204D9C378522B03
:1046100018BF002070470020704700BF686E01205F
:104620002DE9F0410020B4B0FFF7D2FF0024DFF8FD
:10463000A4800546274626464DBB224D2868FFF735
:1046400079FF3B463246CDE900401F4902A805F0FC
:1046500057FE02A801F03BF81C4B1A682B68002B90
:104660000CBF4FF496234FF4B423D21A4FF4704189
:1046700064235343009193FBF1F302A8144905F01E
:104680003FFE02A801F023F834B0BDE8F08169686C
:104690002A6801918B1C1F44D1B2C2F307239C42AC
:1046A000C2F30742009102A84146B8BF1C4605F07C
:1046B00027FE02A801F00BF82846FFF789FF013614
:1046C0000546B9E7686E01206EBD00006C6E0120E2
:1046D00018BD00005ABD000070B50020FFF72AFF8A
:1046E00005460120FFF726FF0C4B1E68B6FA86F43C
:1046F00085424FEA5414B8BF054620461C60FFF7B8
:104700000DFF074A074B002E18BF1346064A691CC7
:104710002046BDE870401360FFF72ABF686E012095
:1047200004B0040004A005006C6E012070B50020E8
:10473000FFF700FF02460120FFF7FCFE1F4E204C52
:10474000054672B968B94FF4D2214FF49620FFF7AD
:10475000CBFE01212846FFF70BFF1A4B3560236083
:1047600029E0AA4208DD00233360164B23604FF492
:10477000B4212368002017E001233360124B23602B
:104780004FF4D221F5E7120E522A08D000B123606F
:104790000E4800F09CFFBDE87040FFF79DBF5A68CF
:1047A000023203EB820301208B4205D21A68551CAA
:1047B000E9D10028D3D170BD2160FCE7686E0120EB
:1047C0006C6E012004B0040004A0050033BD00009D
:1047D00010B50020FFF7FCFE014608B9084610BDE1
:1047E0008478FFF7F5FEDA2C08BF0146F5E70000F4
:1047F0002DE9F04F4FF480729FB0604C6048DFF8B5
:1048000080B1002105F024FA4FF4807200215D4848
:1048100005F01EFAD4F80090B9FA89F84FEA581852
:104820004046FFF77BFE0294574A584C0020B9F1EE
:10483000000F08BF1446FFF7CBFF064626BB4846CD
:10484000FFF778FE411C4046FFF792FE029BB9F14C
:10485000000FC3F800804E4B14BF4FF496224FF464
:10486000B4221C60A21A4FF4704164235343009198
:1048700093FBF1F305A8474905F042FD05A800F0B8
:1048800026FF1FB0BDE8F08F3568C5F30743A3F1DD
:104890000A02092AC5F3072547D81BF8051091BB62
:1048A00010223D48DFF8F0A005F0D2F937463A680B
:1048B000C2F307218D4209D1C2F307410B2927D04A
:1048C00013292CD00A2901D1CAF800703846FFF705
:1048D0007FFE07460028EAD12F4F396881B1204674
:1048E000FFF76AFE0123044657F8231029B120463A
:1048F0000393FFF761FE039B04460133042BF3D1BE
:1049000001230BF805303046FFF762FE064695E7B7
:10491000D2B2022ADADC0AEB82025760D6E7102212
:104920000021504605F094F9D0E7A3F11502082ABA
:10493000E9D8144A525D002AE5D1152B0CBF314647
:10494000002130460368C3F30742152A0FD01D2A01
:1049500008BF0021FFF73CFE0028F3D119B1204623
:10496000FFF72AFE0446074A01235355CBE7C3F35A
:1049700007239D4208BF0146ECE700BF686E012097
:10498000686D0120706E012004A0050004B00400D1
:104990006C6E0120FDBC0000548D0120FFF728BF84
:1049A0002DE9F84FDFF8A8B0274F033392460422D1
:1049B00093FBF2F6DBF80030B41C002B3B684FEAA7
:1049C00084040CBF4FF4B4224FF4D22223449A4201
:1049D00081460D46B84614D2FFF70AFFDBF80030D7
:1049E000002B3B680CBF4FF4B4224FF4D222234477
:1049F0009A4206D2154800F06AFE00273846BDE804
:104A0000F88F2D025FFA8AF141F0A441ADB2D8F8D7
:104A100000700D434FEA094101F47F0129433846F4
:104A2000FFF796FD07F108053146381DC8F800501C
:104A3000FFF78EFD1EB10A9A2846FFF7A5FD083C38
:104A40002544C8F80050D9E76C6E0120D7BC00009F
:104A5000686E012030B59BB0FFF768FE00214FF46F
:104A6000FF621D4805F0F4F8FFF7B2FE1A49002472
:104A7000A0B9194B024653F8301001B10132013090
:104A8000FF28F8D1154901A805F03AFC01A800F06B
:104A90001EFE134800F01BFE1BB030BD0368C3F3BD
:104AA00007420A2A0BD1C3F30722FF2A04D001EBE5
:104AB000C20541F832002B71FFF78AFDD8E7132AAF
:104AC000FAD1C3F30723FF2B1EBF01EBC30241F84A
:104AD00033401471F0E700BFCC830120A3BD000078
:104AE000B7BD00000A4B0022C3F8002101225A6022
:104AF000D3F80021002AFBD00022C3F80C210122A8
:104B00009A60044B0222C3F880211A60704700BFEC
:104B10000010004000E100E0074B0222C3F88020B3
:104B2000064B0022C3F8102101221A61D3F810218C
:104B3000002AFBD0704700BF00E100E000100040F9
:104B400008B504490A780AB1FFF7E6FF00200870AB
:104B500008BD00BF716F01204FF08053586E4000B8
:104B600040F0010070470000024B1868400040F020
:104B700001007047F46F0120024B1868400040F0BC
:104B80000100704724000020024B1868400040F0EC
:104B900001007047F86F012070B504460D461646B7
:104BA000FEF768FA4FF0805301225B6E6270E2708C
:104BB000020A23F00043A271020CE2711A0A0021DA
:104BC00060716372000EA2721A0C1B0E2670A17027
:104BD00025712072E272237370BD000010B5054C80
:104BE000204605F0D3FB01462046BDE81040FEF705
:104BF00022BF00BFFD6F0120104B1B685A1C10B56F
:104C000014D0CBB1012B13D0022B13D0042B13D013
:104C10000B4C0C4A052B08BF1446204605F0B6FB8A
:104C200001462046BDE81040FEF705BF064CF4E7FC
:104C3000044CF2E7054CF0E7054CEEE728000020B5
:104C40004DBE000053BE000048BE00009BB60000F1
:104C500094B6000010B521480278002A3DD14FF0EB
:104C60008043C3F8002101221A60D3F80021002AF2
:104C7000FBD01B4B1B4C00220721C3F80C25C3F8AB
:104C800008151949C3F81025C3F81C15C3F82425C5
:104C90000121C3F82C250822C3F83015C3F81425C8
:104CA000C3F818450224C3F834454FF6FF74C3F81F
:104CB0003C450E4CC3F838451824C3F85445C3F896
:104CC0000423D3F8002242F01002C3F80022084A5D
:104CD000C3F80425FFF706FF017010BD716F0120B6
:104CE0000010004020000402746962752110010068
:104CF000726F0120F8B5104B1B7804460BB9FFF713
:104D0000A9FF0E4E3378ABB10D4A1278D21A02F0D9
:104D100003010C4A02EB411202F1200710685168AE
:104D2000254603C50832BA422C46F7D1013B337001
:104D30000120F8BD1846FCE7716F0120FC6F0120CF
:104D4000706F0120726F012030B5002889B02ADD14
:104D50000D6815F0010426D1042D26D92B6803F027
:104D60000F03092B21D16B683F2B1EDD6846FFF72F
:104D7000C1FFB0B19DF800200435A242A8BF1DF8C4
:104D8000043004F10104A6BF5B0043F001030123DA
:104D9000202C45F8043FF0D1054BDDF809201A60BE
:104DA000042009B030BD0020FBE72046F9E700BF32
:104DB000F86F012030B5384B1B788BB00BB9FFF77B
:104DC00049FF02A8FFF796FF10B900200BB030BDD5
:104DD0009DF808300B2BF8D99DF80930012BF4D140
:104DE0009DF80B30012BF0D12C4D2D4C2D4ADDF8C8
:104DF000111000232B6023709DF80C3013602A4A99
:104E0000116023B9DDF815302B6000230FE0012B72
:104E100011D1DDF815309DF819202B600DF11A0124
:104E20000E239342A8BF134600229A4230D100229B
:104E3000E2540420CAE7022B05D19DF81520122365
:104E40000DF11601EDE7042B0DD10AAA6B4652F8BD
:104E5000130D516803C3DDE9000102F067FE04F0A1
:104E60003DFE2860D1E7052BCFD10AAA6B4652F848
:104E7000130D516803C3DDE9000102F057FE04F091
:104E80002DFE9DF81D2028600A230DF11E01C8E7A4
:104E9000885CA0540132C8E7716F0120F46F0120D3
:104EA000FD6F012028000020F86F012010B5154B80
:104EB0001B7804460BB9FFF7CDFEFFF72DFE124B12
:104EC0000022C3F80445C3F8002101221A60D3F878
:104ED0000021002AFBD00022C3F80C2101229A6095
:104EE000094AD2F80C31002BFBD0084B1978084B3B
:104EF00003EB4113C2F80435FFF70EFEBDE8104086
:104F0000FFF7F0BD716F012000100040706F0120AD
:104F1000726F012000B5002889B01DDD0B6813F009
:104F2000010219D1042B17D9196801F00F010929C1
:104F300012D159683F290FDD043353F8040F10F0E4
:104F4000010118BFC0F347010DF802100132202AF9
:104F5000F3D16846FFF7AAFF002009B05DF804FB13
:104F6000002810B511DD0C68E3070ED56410532C32
:104F70000BD8074B1B780BB9FFF76CFEFFF7CCFD86
:104F8000044BC3F80845FFF7ADFD002010BD00BF7E
:104F9000716F012000100040002810B50DDD0C6875
:104FA000E3070AD56410FF2C07D8054B1B780BB913
:104FB000FFF750FE034BC3F82445002010BD00BF8F
:104FC000716F012000100040002813B515DD0C683A
:104FD000E10712D564100A4A0A4B072CCDE90023D9
:104FE0000BD8094B1B780BB9FFF734FE02AB1C44FE
:104FF000064B14F9082CC3F80C25002002B010BD94
:10500000E2ECF0F4F8FC0004716F012000100040A5
:1050100070B5002888B020DD086810F001041CD1AC
:1050200004281AD9036803F00F03042B15D1FEF7E7
:10503000E5FA064605F0AAF9122828BF122005460F
:1050400000F10D0202216846FFF7A6FD8DF80D5014
:10505000A54205DC6846FFF729FF002008B070BDB7
:105060000DEB0403325D9A730134F1E72DE9F04151
:10507000012888B00D4630DD086810F001042CD1FD
:1050800004282AD9036803F00F03042B25D14B68A9
:10509000DB0722D5FEF7B2FA804605F077F96D6896
:1050A0000E2828BF0E206E10074600F111020121C4
:1050B0006846FFF771FD6B128DF80D606D14360EAA
:1050C0008DF80E308DF80F508DF810608DF811703E
:1050D000A74206DC6846FFF7E9FE002008B0BDE8FD
:1050E000F0810DEB040318F804209A740134EFE703
:1050F00030B5002889B016DD0C68E30713D56510BC
:10510000684610220021FFF747FD63128DF80D500D
:1051100064142D0E68468DF80E308DF80F408DF812
:105120001050FFF7C3FE002009B030BD174BD3F875
:10513000002122B10022C3F8002101229A60D3F895
:105140000C2102B30021C3F80C11D3F80024012A6A
:105150000F4A19D1D3F848355B4213600D4A1378D2
:10516000032B9CBF013313700B4A1378013303F0F8
:1051700003031370094A02EB4313044AC2F80435CF
:10518000024B01229A6070471160F9E7001000405D
:1051900024000020FC6F0120706F0120726F01203D
:1051A000024A0348102100F07DB800BFC8BD0000CE
:1051B000BFBD0000044A05491368C8540133C3F356
:1051C00009031360704700BF2C7401202C7001206C
:1051D00070B51149114A0B68834202DC00230B6051
:1051E00017E0855CA5F1FA06012E00F1010405D84F
:1051F0009C420FDAA55C013D1F2D01D92046EBE74B
:105200000446151A165D2E550134A342FADC181A0D
:10521000086070BD1570FAE73878012038740120F5
:1052200008B5FDF71FFF074B1A68824284BF0022B2
:105230001A601B68C01A44F62063984294BF00208D
:10524000012008BD2870012070B5094C094D0A4E97
:1052500023682A68934200D170BDF05CFEF764F9C0
:105260000028F9D023680133C3F309032360EFE773
:10527000307401202C7401202C70012070B5074E71
:10528000074D044633682A689B1ADB43C3F30903BE
:10529000A34200DB70BDFFF7D7FFF3E72C740120BA
:1052A00030740120F0B5074D2B680B2B08DC064F3E
:1052B0000C245C433E19C6E90112013338512B60BE
:1052C000F0BD00BF34740120648D012008B5FCF7E7
:1052D0004BF8FFF7FFF8FCF76BF8FEF7B7F8FEF7AF
:1052E00065FDFEF78DFDFFF75BFF00F0F1FF01F0BC
:1052F00005FABDE8084001F039BC000008B54FF4DC
:1053000016620021034804F0A3FC034B00221A603C
:1053100008BD00BF6C7A01209C050020064B074A9F
:105320001B6812689B1ADB43C3F309038342D4BF93
:1053300000200120704700BF2C7401203074012030
:10534000F8B507460E4614461D4673B90320FFF70D
:10535000E5FF10B3FA20FFF72DFFF8B2FFF72AFFA1
:10536000F0B2BDE8F840FFF725BF501DFFF7D6FFAC
:1053700098B1FB20FFF71EFFF8B2FFF71BFFF0B25A
:10538000FFF718FFE0B2FFF715FFC4F30720FFF7A0
:1053900011FF2E46731B9C4200DCF8BD16F8010B72
:1053A000FFF708FFF6E70000F8B50C4E0C4D00249F
:1053B000F0273368A34203DCBDE8F840FFF79EBF47
:1053C00007FB04F359195B5D2BB100231A4649789A
:1053D0001120FFF7B5FF0134EBE700BF9C0500206B
:1053E0006C7A0120F8B50E4C0E4E07460025BC42E3
:1053F00005F1010511D0237853B100231A466178D5
:105400001120FFF79DFFF0220021204604F020FC30
:105410000A2D04F1F004EAD1F8BD3560F8E700BFC9
:105420006C7A01209C0500202DE9F04F12F0010656
:10543000ADF54F7D82468B4617D001238DF8143091
:1054400042FA03F354128DF8153052141B0E8DF8E6
:1054500017208DF818308DF8164005AB0522FFF7A0
:105460006FFF0DF54F7DBDE8F08F042A1FD911683D
:1054700001F00F03042B2BD105AD022310462B7036
:10548000FEF7BCF8044604F081FF40F2233290425C
:1054900028BF1046621EB04204DC2B46421C59460F
:1054A0005046DCE7013612F8013FAB55F3E740F018
:1054B000C880A2F1040CDCF100024FF0030342EBC0
:1054C0000C028DF814308DF8152005AB0222E6E7AA
:1054D000092B40F09180154604238DF8143055F8BF
:1054E000043F4FEA6308B8F1200F8DF815804FEAAA
:1054F0006323A8BF4FF020088DF816308DF8178071
:1055000006AC03220521B04502DC05ABE21AC6E772
:1055100055F8040F10F0010706D1042847D9036895
:1055200003F00F03022B0DD14FF001032370431042
:10553000637047121B0E4014A770E070237105348E
:105540000136E0E7042B30D123464FF0020C03F87C
:1055500002CBCDE9012100930393FEF74FF881467A
:1055600004F014FF0C28DDE901210AD8009B6070CB
:10557000874201D1DC19E3E719F80740DC55013710
:10558000F6E723460C2003F8010F09F1FF3009F17B
:10559000080910F8017F03F8017F4845F9D12E234F
:1055A000E372237363730E34CAE7012B08D12346D9
:1055B000071F03F8022B7842784160701C46BFE752
:1055C000092B09D1042323704368581060705B12C3
:1055D000A370E7700434B3E7032B0AD1217003688A
:1055E000C3F30F10C3F34173C3EB800363701B124B
:1055F000EEE727700134A3E7032B7FF432AF0523D6
:105600008DF81430C1F30F13C1F34171C1EB830165
:105610000B1264298DF816300B46A8BF64238DF851
:1056200017308DF815100332DBB29E4202DB05AB5A
:105630000A1D34E705A8304412F8014F0471013601
:10564000F3E7002A7FF40DAF33E700000F4970B590
:10565000F022002402FB04135D78854203D001345C
:105660000A2CF7D170BDF0221846002104F0F0FAA0
:10567000074A1368013BA34200D114600023294666
:105680001A461120BDE87040FFF75ABE6C7A01201F
:105690009C05002030B5B3B032AC0223054604F8B7
:1056A000C83D04F073FEC72828BFC720691E002329
:1056B000984207DC421C2346FE211420FFF740FEDF
:1056C00033B030BD013311F8012FE254F0E770B56B
:1056D000B2B032AC0223054604F8C83D04F056FED1
:1056E000C72828BFC72006460023681E9E420BDC41
:1056F00006F13200FFF7C2FD2346721CFF21142081
:10570000FFF71EFE32B070BD013310F8012FE254D6
:10571000ECE700002DE9F04F0128B9B0814688463A
:1057200003DC1B20FBF714FF58E00868C2072BD4EA
:10573000042829D9036803F00F03042B24D1FDF7B3
:105740005DFF0546D8F80400C3071FD404281DD9FF
:10575000036803F00F03042B18D1FDF74FFF064633
:10576000214BDFF890A01B6803930027039BBB42EB
:105770000EDC00962B461D4AC82106A804F08CFDBD
:1057800006A8FFF7A4FFCCE7194DDBE7184EE7E7C3
:105790000C2303FB07F202EB0A03294652F80A0026
:1057A000049304F0E9FD049B044618B9D3E9013BD6
:1057B0009C4201DB0137D9E70BEBC40231465BF8B1
:1057C00034000593049204F0D7FDDDE9042340B9C9
:1057D000536808F10801A9F10200984739B0BDE803
:1057E000F08F0134E4E700BF3474012024BF0000CF
:1057F0009FB70000648D01202DE9F0411F4F204A22
:10580000D7F8008005460023F02098450EDC0024E0
:10581000F02000FB04F15318565C8EB101340A2CC1
:10582000F7D11848BDE8F041FFF751BF00FB03F185
:1058300054186478AC4201D1515CE9B90133E4E712
:10584000F0223146184604F003FA0F49457051F82A
:10585000351085700222A0450270C0E90212C0E92D
:10586000046601DC01343C60002329461A461020FE
:10587000BDE8F041FFF764BDBDE8F0819C05002064
:105880006C7A01206DC30000CC83012070B5FFF756
:105890008BFD094EFF246FF0070505FB046393F8A9
:1058A000FC37043B012B03D8E043C0B2FFF7A4FF51
:1058B000013CF2D170BD00BFCC8301202DE9F8433B
:1058C0001D4E07460D460024B046E3009A19127992
:1058D000062A01D0032A23D158F80300836803F075
:1058E0007F031C2B1CD1C36803F07F02042A17D14D
:1058F000026902F07F02192A12D11B0A00EB830011
:105900001030FDF77BFE0378814633B104F03EFD95
:10591000A84205D100239D4207DCE0B2FFF76CFFEF
:105920000134FF2CD1D1BDE8F88319F80310FA5CDB
:105930009142F5D10133EEE7CC830120F8B5094F50
:105940000546FF246FF0070606FB047393F8FC3747
:10595000AB4203D1E043C0B2FFF74EFF013CF3D1AD
:10596000F8BD00BFCC8301202DE9F84FFDF77AFB8D
:10597000584B1A68824284BF00221A601A6842F2A9
:105980000F71821A8A420BD95349186000235A18A2
:105990001279073A022A0FD90833B3F5FF6FF6D10F
:1059A000BDE8F88F0720FFF7C9FF8AF800802EE0D6
:1059B0000820FFF7C3FF3FE0FDF75CFB002814BFA2
:1059C000044601240020FDF781FC81460020FDF7FC
:1059D00091FC424D424E0746B9F1000F17D02B689B
:1059E000002B70D133682C60002B6FD0DFF8F8B03B
:1059F000DFF8F0A09BF800304FF00108002BD1D168
:105A00000920FFF79BFF8AF800808BF80080AFB178
:105A100033689BB92B6834601BB3DFF8C8B0DFF87C
:105A2000C8A09BF800304FF00108002BC0D109201E
:105A3000FFF784FF8BF800808AF800802B6883B121
:105A4000284A1178904661B99C4238BF2C602B6877
:105A5000E31A312B05D90720FFF770FF012388F8DF
:105A60000030326882B1204B1978984661B9A24261
:105A700088BF34603368E41A312C05D90820FFF759
:105A80005DFF012388F800302B685BB1B9F1000F8E
:105A900008D1144C227812B90720FFF74FFF0023DA
:105AA0002B6023703368002B3FF47AAF002F7FF414
:105AB00077AF0D4C227812B90820FFF73FFF002383
:105AC000336023706CE7002FA2D1B9E7002FA1D17A
:105AD000B4E700BF24700120CC83012014700120A2
:105AE0001C700120187001202070012037B5054678
:105AF000FFF75AFC02A8002440F8044DFDF7CEFB46
:105B000021462046FEF7E4F9FEF75EFCFDF77AFC3D
:105B1000FDF794FCFEF7DAFCFDF7C8FA25B1FDF7B6
:105B20001DFD0248FFF7D3FD03B030BD5EC300008A
:105B3000002301461A461120FFF702BC07B51312D5
:105B40008DF801208DF802301314120E8DF800101C
:105B50008DF803308DF8042001466B460522132092
:105B6000FFF7EEFB03B05DF804FB0A460146122086
:105B7000FFF75ABC70B50C46054601F13200FFF73D
:105B80007DFB2B46224600211B20BDE87040FFF71D
:105B9000D7BB10B4144603460A46142021465DF8CC
:105BA000044BFFF7CDBB000030B5084C01444FF06B
:105BB000FF33884201D3D84330BD10F8015BDAB21D
:105BC0006A4054F8222082EA1323F2E740BF000023
:105BD000FE2837B5044614D80B4B53F8300080B17B
:105BE000416808308900FFF7DFFF02AD45F8040D7A
:105BF0000920FFF743FB2B46042221461720FFF71D
:105C00009FFB03B030BD00BFCC830120F8B5074631
:105C1000FEF7DEFD4FF0FF3504460CB92846F8BD0F
:105C20002668C6F30743152B0CD104F1080138464A
:105C300004F0A2FB08B9C6F307252046FEF7C8FC0E
:105C40000446EAE71D2B08BF4FF0FF35F5E70000DB
:105C50002DE9F047BD4CBE4D9CB0FFF7F5FA20682A
:105C6000C0F580612844FDF747FC236803440646DD
:105C700023607BB1B74F002E0FDC2B78FA2B40F05E
:105C800025812368022B16DCFFF7CAFA10B1012028
:105C9000FFF79EFA1CB0BDE8F0872068C0F5806170
:105CA0002844FDF729FC2368034406462360FDF7DA
:105CB000D9F93860DFE76B78AC78023B182B2CD829
:105CC000DFE813F019002D003100350038004100E5
:105CD0002B004B0080008A008E00A400E000F10041
:105CE0002B002B002B002B002B002B002B002B005C
:105CF0002B002B00FF00FF2C0FD02046FFF7A6FC47
:105D0000954A002342F8343002EBC4022146137155
:105D1000132000931A46FEF743FE0320B8E72046FF
:105D2000FFF76AFDF9E72046FFF790FCF5E7FFF77C
:105D3000ADFDF2E7FFF738FB0020FFF7D7FE8748FD
:105D4000FFF7C5FCE9E7632CE7D8854B214653F8FC
:105D500024201520FFF768FBDFE7FEF739FD6FF021
:105D600007080446002CD8D02768C7F30743152B33
:105D700004D02046FEF72CFC0446F3E704F10806A5
:105D8000304604F003FB05460530FFF777FAFB20A9
:105D9000FFF710FA1D20FFF70DFAC7F30720FFF7F2
:105DA00009FAE8B2FFF706FAC5F30720FFF702FA8F
:105DB000A8EB0407F3199D42DBDD16F8010BFFF792
:105DC000F9F9F7E7002300931A4619461D20FEF75C
:105DD000E7FDFDF7C3FBA0E72046FFF7F9FE9CE7D0
:105DE000FDF750F95F4A009064215F4B03A804F06F
:105DF00053FA022303A88DF80C3004F0C7FA03AB62
:105E0000024600211620FFF79BFA86E7524F002535
:105E100057F8354007EBC5035CB3D4F8048093F81A
:105E200004A04FEA8806B01DFFF728FAFB20FFF711
:105E3000C1F9012006F10109FFF7BCF9E8B2FFF74B
:105E4000B9F95FFA89F0FFF7B5F9C9F30720FFF751
:105E5000B1F95046FFF7AEF9083404EB0609A14545
:105E60000BD8FFF7F1F906EB080001F049FCFFF74A
:105E7000EBF90135FF2DCBD14FE714F8010BFFF7FC
:105E800099F9ECE70024FFF78FFA224621460094A7
:105E90002346DA20FEF784FD4FF4FF6221462E48A8
:105EA00003F0D6FE95E7012C02D1FEF7B9FB34E7EB
:105EB000022C02D1FEF772FD2FE70120FFF716FE3C
:105EC0002BE700231A4621461A209CE7FB2B7FF480
:105ED000DEAE2268042A7FF7D7AEB5F8037040F231
:105EE000F6339F423FF7D3AE3B1D9A427FF7CCAECD
:105EF000EB5CFE2B7FF4CBAE6B78AC781B2B07F101
:105F0000FF3673D01AD8072B57D0082B30D0012B6F
:105F100019D1FF2C17D02046FFF798FB6D79134B52
:105F200000932146BB1E2A460A20FEF739FD0A4B84
:105F300043F8340003EBC404257104E01D2B67D043
:105F400059D31E2B7CD0781DA2E600BF38780120E3
:105F50003874012028700120CC83012040C3000048
:105F6000C48B012057C3000052C300003E740120BF
:105F7000632CE8D86B79022B0CD0032B14D0012BA7
:105F8000E1D1D5F80630364A5B0043F0010342F810
:105F90002430D8E7002ED6DDB91E3248FDF74BFD80
:105FA0002F4B43F82400CEE7AB79002B2C4B0CBFD2
:105FB0000022042243F82420C5E7632EC3DC3246C6
:105FC000294903A803F020FE1CAB1E4403A80023AC
:105FD00006F8643CFFF71AFE0028B4DB204B21468C
:105FE00053F820201520FFF71FFAACE731461E4872
:105FF000FFF764FCA7E7FF2CA5D06A79022AA2D894
:10600000184B00932146BB1E0B20FEF7C9FC9AE7F4
:10601000632EA8BF6326002303A9B3420BDB1CAA8F
:1060200026EAE6731344002203F8642C152000913D
:10603000731C2146E9E7EA185279CA540133ECE7A8
:10604000012C80D1002E7FF77EAF6B791BB1322BF4
:10605000A8BF32231C4664235C43044B1C6072E7D8
:10606000C48B01203E7401203D74012004000020F7
:10607000084B01221A60084A1368002BFCD0074B1A
:106080001868042390FBF3F00638400040F001004C
:10609000704700BF00C0004000C1004008C500407C
:1060A0000120704710B5064C204600F08BFE0549D4
:1060B000204600F0EDFE044B01221A6010BD00BF27
:1060C00074780120801A06003C78012010B5064C37
:1060D000204600F077FE0549204600F0D9FE044B2B
:1060E00001221A6010BD00BF30790120801A06001D
:1060F0004078012010B501210D20FCF7C9FF094CA3
:1061000001210E20FCF7C4FF00210F20FCF7C0FF87
:10611000204600F099FD20461021BDE8104000F017
:10612000A9BD00BF547801202DE9F8430C68E307AE
:1061300004D40D20BDE8F843FBF70ABA64102FD44D
:10614000FCF7A4FFA0422BDB00212046FCF7A0FFB8
:106150004FF4FA620121204601F00AFB00B3DFF898
:106160006C8000254FF00109002707264FF47A7252
:106170000121204601F0FCFA90B12828C4BF09FA99
:1061800006F31F4316F1FF36F0D205F8087001350B
:10619000052DE9D1012206210920FDF7CBFB08B925
:1061A00000200FE003460B2243F8042F064900F1BC
:1061B000180411F8012F520042F0010243F8042F95
:1061C0009C42F6D1BDE8F883437801204478012051
:1061D00010B50468E30704D40D20BDE81040FBF7B8
:1061E000B7B96410FF2C01D91720F6E7FFF782FF3B
:1061F000E1B2024800F061FD002010BD547801209A
:1062000008B5FFF777FF0021034800F056FD400076
:1062100040F0010008BD00BF54780120274A82B039
:1062200001210023ADF80630C2F8F015C2F80015C0
:1062300019461A0102F1804202F5E0420133082BAF
:10624000C2F81415C2F81015F3D11C4B4FF4E062DC
:10625000C3F818250422C3F81425C3F810250DF13E
:106260000602C3F82C260122C3F830261A60D3F8A0
:106270000021002AFBD00022C3F8002101225A602D
:106280000E4B1A46D3F804110029FBD00021C3F8A5
:10629000041101219960D2F81431002BFBD00020A9
:1062A000C2F81401C2F80005BDF806301BB28342E3
:1062B000C8BFA3F50B70400002B0704700700040EB
:1062C00008B5FFF7ABFF400040F0010008BD00003B
:1062D000024A03480A21FEF7E5BF00BF84C300005D
:1062E000D4C3000070B50668F10705D54568EA0714
:1062F00002D58468E30704D40D20BDE87040FBF7A5
:1063000027B97610802E01D91520F6E76D10FF2DE4
:1063100001D91620F1E76410FF2C01D91720ECE712
:106320000A4B1B680BB9FFF7BDFEF1B2084800F03D
:106330002DFEE9B2064800F00DFDE1B2044800F080
:1063400009FD034800F08DFE002070BD3C7801205F
:10635000747801200C4B1B6870B506460D46144638
:106360000BB9FFF7B3FEF1B2084800F00FFEE9B237
:10637000064800F0EFFCE1B2044800F0EBFC0348F3
:10638000BDE8704000F06DBE4078012030790120FA
:106390000128F8B536DD0D68EA0733D51A4B4C688D
:1063A0001B686D100BB9FFF77DFEE9B2174800F0CE
:1063B000EDFD14F001050DD0C4F34701134800F0C2
:1063C000C9FC124800F04DFE18B12320FBF7C0F8BD
:1063D0000020F8BD042CF4D9236803F00F03092B27
:1063E000EFD154F8046F094F7610AE42E9DD54F84E
:1063F000041FCB0704D5C1F34701384600F0AAFCBF
:106400000135F2E70120E4E73C78012074780120AF
:1064100038B50468E20702D54568EB0704D40D20BF
:10642000BDE83840FBF794B86410802C01D91520E2
:10643000F6E76D10FF2D01D91620F1E7124B1B680E
:106440000BB9FFF72FFEE4B22146104800F09EFD85
:10645000E9B20E4800F07EFC00210C4800F0A0FDDF
:1064600020B14042400040F0010038BD01222146E9
:10647000064800F088FD054800F063FC0028F1D0D4
:10648000024800F061FCEDE73C78012074780120BF
:1064900038B5124B1B6804460D460BB9FFF716FEC4
:1064A000E4B221460E4800F071FDE9B20C4800F05C
:1064B00051FC0B4800F0D5FD08B1404238BD012227
:1064C0002146074800F05FFD054800F03AFC00282F
:1064D000F4D00348BDE8384000F036BC40780120D5
:1064E00030790120F8B5354E354D376804466FB91F
:1064F0000D211D20FFF7CCFF5A2816D101222A704A
:106500002A211D20FFF726FF0123336095F9003073
:10651000022B29D0032B44D0012B45D121461D202D
:10652000FFF7B6FF4FF0FF3424E00F211920FFF7EB
:10653000AFFF332805D102232B705F2220211920C1
:10654000E0E70D211E20FFF7A3FFC7280AD1032390
:106550003A462A211E202B70FFF7FCFE1B222A211F
:106560001E20CFE72F70CFE7012C13D1292119204E
:10657000FFF78EFF7F28C8BFA0F580706FF07E0305
:106580009842B8BF1846C82358437F2390FBF3F0C6
:106590006043F8BD032C0BD12B211920C0E72D211E
:1065A000FBE721461E20BBE74FF0FF340020EAE75F
:1065B000052CF4D04FF0FF340020DFE74C780120A9
:1065C0002C00002008B50120FFF78CFF400040F0B0
:1065D000010008BD08B50320FFF784FF400040F02C
:1065E000010008BD08B50520FFF77CFF400040F022
:1065F000010008BD38B5104B1B6813B90120FFF727
:1066000071FF0120FFF76EFF04460320FFF76AFFCA
:1066100005460520FFF766FF6D4304FB045400FBAD
:10662000004002F041FF01F09FFB03F057FA4000E9
:1066300040F0010038BD00BF4C7801200128F8B5BA
:1066400035DD0F68FB0732D54D6815F001062ED1F8
:10665000042D2CD92B6803F00F03092B27D16C686C
:10666000144B64101B68202CA8BF20240BB9FFF723
:1066700019FDC7F3470122460F480F4F00F083FC76
:106680000435A64211DA0C4800F05BFB18B9700023
:1066900040F00100F8BD384600F056FB400040F0E5
:1066A000010045F8040F0136EBE76000F0E7012038
:1066B000F0E700BF3C78012074780120002070478B
:1066C000012070470020704700207047012070476C
:1066D000002070470020704700207047002070475E
:1066E000002070470020704700207047002070474E
:1066F000002070477047704770470000024A034807
:106700000E21FEF7CFBD00BF38C40000A8C40000B2
:106710000246104601320378013B1F2BF9D970471E
:1067200008B5FFF7F5FF0378002B39D0222B00F1D5
:10673000010011D1037823B1222B00F1010204D111
:106740001046BDE80840FFF7E3BF5C2B02D1437859
:1067500003B1821C1046EDE73A2BF2D02C2BF0D07F
:106760007B2B0BD1FFF7D4FF0378002BE9D07D2BD7
:1067700001D10130E5E7FFF7D3FFF5E75B2B10D040
:106780000246104612F8013B002BDAD0202BD8DD50
:106790002C2B05D003F0DF015D2901D0222BF0D195
:1067A00008BDFFF7B5FF0378002BCAD05D2BE0D002
:1067B000FFF7B6FFF7E708B5F0B1FFF7A9FF0378D9
:1067C000222B1AD07B2B1AD05B2B1AD0A3F13002CC
:1067D000092A05D92D2B05D14278303A092A07D844
:1067E000032009E0742B0ED0662B0ED06E2B0ED03A
:1067F000181C18BF0120404208BD0420FCE70220FD
:10680000FAE70120F8E70520F6E70620F4E707207D
:10681000F2E738B5FFF77CFF03782D2B11D101305B
:106820004FF0FF34431E00210A2501E005FB012142
:1068300013F8012F303AD0B20928F7D904FB01F040
:1068400038BD0124EEE710B51446FFF761FF037869
:10685000222B02D000230B7010BD621E0130037882
:10686000222BF7D0002BF5D05C2B07D0441C002A3C
:10687000F0DD01F8013B013A2046F0E74378622B56
:1068800000F1020409D0662B09D06E2B09D0722BBF
:1068900009D0742B08BF0923E9E70823E7E70C2395
:1068A000E5E70A23E3E70D23E1E710B50446FFF728
:1068B00037FF0346A342184604D90278202A03F181
:1068C000FF33F7D910BD08B590B1037883B1FFF756
:1068D0001FFF037803F0DF035D2B09D0FFF720FFD4
:1068E00003782C2B08BF0130BDE80840FFF710BF2C
:1068F000002008BD38B50D1E0DDD03785B2B0AD1D5
:106900000130FFF705FF0124A54205D0FFF7DBFFAB
:1069100010B10134F8E7002038BD38B5154609B18B
:1069200000230B70F8B10378E3B1FFF7F1FE0378B1
:106930002C2B044603D10130FFF7EAFE04462378EE
:106940007D2B0FD019B12A462046FFF77CFF204649
:10695000FFF7E6FE03783A2B05D10130BDE8384059
:10696000FFF7D6BE002038BD2DE9F0410D469AB0A4
:1069700004462F789FB32E21284603F0F0FC804672
:1069800090B1461B303F092F13D82846FFF741FF2F
:1069900001462046FFF7AEFF044604B3B8F1000FEE
:1069A0001DD001363544E4E7284603F0EFFC0646E7
:1069B000E8E723787B2B11D1601C642201A9FFF743
:1069C000ACFF044658B13246294601A803F0E6FC64
:1069D0000028E2D02046FFF7A3FEEEE70024204681
:1069E0001AB0BDE8F08138B50D1E04461CDDFFF776
:1069F000E2FE012807D1601C012D00D138BDFFF750
:106A000062FF013DF8E702280ED100221146601C0A
:106A1000FFF783FF012DF1D0FFF755FF002211464C
:106A2000FFF77BFF013DF5E70020E7E7F8B50C1E17
:106A3000074615461E4613DDFFF7BDFE02280FD19F
:106A400032462946781CFFF768FF012C00D1F8BDBB
:106A5000FFF739FF32462946FFF75FFF013CF4E7B5
:106A60000020F4E710B50446C8B1FFF751FE0378E3
:106A70007B2B0AD10130002400221146FFF74DFF85
:106A800068B1FFF74DFE0134F6E75B2B06D101300C
:106A90000024FFF718FF10B10134FAE70024204664
:106AA00010BD002870B514DD0D68EB0711D56D1011
:106AB000013DFDF78DFE00264FF0FF3460B916B39F
:106AC000304603F063FC01463046BDE87040FCF7F9
:106AD000B2BF4FF0FF35ECE70368C3F30742152A56
:106AE0000BD1C3F307239C42B8BF1C469D4201D182
:106AF00000F10806FDF76CFDE0E71D2A04BF002643
:106B00004FF0FF34F6E7601C400040F0010070BD1C
:106B100010B508680C46FCF771FDFFF777F8002800
:106B2000A2BF034B626843F82020002010BD00BFC5
:106B3000C48B012008B50868FCF760FDFFF766F814
:106B40000028AABF024B012053F8200008BD00BF57
:106B5000C48B012008B50868FCF750FDFFF756F814
:106B60000028ACBF0420002008BD0000024A0348F2
:106B70000421FEF797BB00BF38C5000031C50000F7
:106B800008B5FCF76DFCFCF70DFDFEF79FFB044814
:106B9000FEF79DFDFDF75EFFBDE80840FEF776BEFF
:106BA00087C50000FCF73CB938B50025057329B945
:106BB0000B4B0C4A0C48232102F0B8FF01600B4933
:106BC00051F82220027151F8233083719DF8103062
:106BD00051F8233043710223C371856038BD00BF73
:106BE0009FC500001FC60000ADC500007CC60000A8
:106BF000037B23B9437383730361012303737047DA
:106C000084B00DF1100C0CE90E009DF8081002681C
:106C100000230129C2F80035039B12D00BD30329AE
:106C20000CD0C2F85435019BC2F824350123C2F8B8
:106C3000003504B0704743F00203F2E743F0040369
:106C4000EFE743F00603ECE710B5FFF7D1FF036869
:106C50008279C3F808254279C3F80C250279C3F874
:106C60001025034BBDE810400ECBFFF7C9BF00BF96
:106C7000687801200A0611D43F2912D81F2913D899
:106C80000F2914D8072915D803298CBF4FF080434A
:106C90004FF000430268C2F8243570474FF000738C
:106CA000F8E74FF08063F5E74FF00063F2E74FF04D
:106CB0008053EFE74FF00053ECE70368C3F81C156F
:106CC000D3F80821002AFBD0D3F818050022C3F816
:106CD0000821C0B27047000007B5094B09490A48AE
:106CE0004FF080421A6000229A6002221A710F232C
:106CF00000930E220D23FFF757FF03B05DF804FB4E
:106D00006878012000300040547801202DE9F843D4
:106D100080460D46174601EB02090C464C45A4EB94
:106D200005060BD0D8F8003014F8011B1B6840464C
:106D300098470028F2D13046BDE8F8833E46FAE78E
:106D40007047203000F03CBA203000F02BBA2030E1
:106D500000F03CBA38B5437F0D460BB9002038BD72
:106D600000F16804204600F039FA0028F6D12046E8
:106D7000294600F008FA0120F1E700002DE9F04172
:106D80001E4600254FF47A73C0E901530C4B0446AC
:106D900040F8203B8846174600F0ECF904F1680003
:106DA00000F0E8F99DF8183063769DF81C302676DF
:106DB000C4E90487A37665772046BDE8F08100BF6B
:106DC00064C60000F0B5837E2E4C2F4D0121C176A4
:106DD00054F82320437E54F8233012F0200F14BFC0
:106DE0002F464FF0A04702F01F0213F0200F03F0D0
:106DF0001F0308BF4FF0A04502F5E07203F5E073F2
:106E000040F20C6647F8226045F8236003694FF0B2
:106E1000CC72C3F8242503690622C3F80025827EBC
:106E2000036954F82220C3F80825427E036954F808
:106E30002220C3F80C2590F91830144A5C0903F09D
:106E40001F03994004F1600342F8231090F91830B1
:106E5000002BBDBF03F00F0302F6FC32D2189B18C3
:106E6000B5BF40234022137683F8002390F91830F1
:106E70000122590903F01F0302FA03F3034A42F8FF
:106E80002130F0BD7CC600000003005000E100E0AE
:106E9000C37EA3B103690022C3F800250A4B9942BF
:106EA0000ED90A4B994294BF4FF080614FF0C861F0
:106EB0000369C3F8241503690622C3F80025704747
:106EC0004FF0CC71F4E700BFA086010090D0030022
:106ED0002DE9F041044688461F461546002A50D049
:106EE00000F12006304600F059F92369C3F888857F
:106EF000236901221A622369C3F834652369C3F840
:106F0000385523691A602269D2F84C311BB9D2F87E
:106F10002431002BF8D00023C2F84C312269D2F87A
:106F20005C311BB9D2F82431002BF8D00023C2F811
:106F30005C3122696FB9D2F8243153B90123D3618E
:106F40002369D3F84821002AFBD00022C3F8482146
:106F500009E0012353612369D3F80421002AFBD0FF
:106F60000022C3F804212369D3F8242112B100229E
:106F7000C3F824212369D3F83C052066C0B2BDE8DC
:106F8000F0811046FBE70123FFF7A2BF10B50446CE
:106F900080F8B010683000F001F90123637710BD6C
:106FA000F8B500234377036990F8B020C3F888252B
:106FB000036901261E62036900F168050446C3F8EF
:106FC000445528460F4600F0FBF82369C3F84805EE
:106FD00023699E602369D3F850211AB9D3F824217C
:106FE000002AF8D00022C3F85021284600F0E8F823
:106FF000236930B1D3F860211AB9D3F82421002ACB
:10700000F8D00022C3F8602123696FB9D3F8242196
:1070100052B90122DA612369D3F84821002AFBD052
:107020000022C3F8482109E001225A612369D3F8FC
:107030000421002AFBD00022C3F804212369D3F8DD
:10704000240168B10022C3F824212369D3F8C404C1
:10705000C3F8C404022803D004280CBF0320042072
:10706000F8BD0121FFF79CBF70B54369D3F86421D7
:10707000044692B10022012500F12006C3F86421E4
:107080000577304600F08AF86369C3F834656369B0
:107090004022C3F8382563691D636369D3F868210A
:1070A000DAB10025C3F8685104F16806012363775B
:1070B0002577304600F072F8D4F8B43003B1984721
:1070C000636965773046C3F8446500F079F8636911
:1070D000C3F84805636901225A636369D3F8042140
:1070E00062B10022C3F80421237F3BB16369D3F866
:1070F0003C05D4F8B830206603B198476369D3F8EB
:10710000242152B10022C3F824216369D3F8D0248A
:10711000C3F8D024636901225A6170BD0148FFF7AA
:10712000A3BF00BF747801200148FFF79DBF00BFD7
:107130003079012007B514231322CDE900320A4A21
:107140000A4811460323FFF719FE4FF040221E2381
:107150001F21CDE90031064804231146FFF70EFE3A
:1071600003B05DF804FB00BF0030004074780120DC
:107170003079012008B54022002102F069FD00228B
:10718000C0E9102208BD026C10B5531C446C03F01A
:107190003F039C421CBF8154036410BD0023C0E91F
:1071A00010337047D0E9102393421FBFC25C0133F4
:1071B00003F03F03436414BF10464FF0FF307047A5
:1071C000D0E91030181A48BF40307047D0E910237A
:1071D000934214BFC05C4FF0FF307047036C406CAB
:1071E000013303F03F031B1A584258417047000017
:1071F0000649074A074B9B1A03DD043BC858D05089
:10720000FBDC00F04DF8F9F71BF9000024CB00007F
:107210000000002034020020FEE7FEE7FEE7FEE764
:10722000FEE7FEE7FEE7FEE7FEE7FEE7094B1B7819
:10723000062B0CD1084B1B681A0708D1074B18689E
:1072400000F0F000A0F13003584258417047002090
:10725000704700BFE00F00F0E40F00F0E80F00F00F
:107260000C4B1B78062B10D10B4B1B681A070CD14B
:107270000A4B186800F0F003302B08D000F0E00053
:10728000A0F1400358425841704700207047012048
:10729000704700BFE00F00F0E40F00F0E80F00F0CF
:1072A00008B5FFF7C3FF10B14A4B4B4A1A60FFF70E
:1072B000D7FF28B1494B4A4A1B68C3F342331360D6
:1072C000FFF7B4FF20B1474AD36823F08073D3603F
:1072D000FFF7C6FF40B14FF080430022C3F80C21F6
:1072E000C3F81021C3F83825FFF7A0FF10B13E4BBB
:1072F00003221A60FFF79AFF40B13C4B05221A6047
:1073000001229A6700229A603F225A60384B1B780C
:10731000062B50D1374B1B681B074CD1364B1B68D3
:1073200003F0F003502B46D14FF08052334BD2F88C
:107330000414C3F82015D2F80814C3F82415D2F8A1
:107340000C14C3F82815D2F81014C3F82C15D2F871
:107350001414C3F83015D2F81814C3F83415D2F841
:107360001C14C3F84015D2F82014C3F84415D2F801
:107370002414C3F84815D2F82814C3F84C15D2F8D1
:107380002C14C3F85015D2F83014C3F85415D2F8A1
:107390003414C3F86015D2F83814C3F86415D2F861
:1073A0003C14C3F86815D2F84014C3F86C15D2F831
:1073B0004424C3F87025124AD2F8883043F470038D
:1073C000C2F88830BFF34F8FBFF36F8F0D4B0E4A5B
:1073D0001A6008BD74C007400DF0ADBA4402001039
:1073E0003C050040F0ED00E0A005004010560040D4
:1073F000E00F00F0E40F00F0E80F00F000C00040E4
:1074000000ED00E0300000200090D0030120704724
:1074100003681322DB69184770470369C3F81C151A
:107420000369D3F81C21002AFBD00022C3F81C21D9
:107430000120704710B490F95C30144C59090122B6
:10744000203103F01F0302FA03F344F821300369EB
:107450005DF8044B0421C3F8081303695A600369FB
:10746000DA6003690022C3F8002502694FF0FF3398
:10747000C2F80C350269C2F814350269C2F8083541
:1074800002691430C2F81035FFF788BE00E100E051
:107490001430FFF795BE1430FFF798BE1430FFF795
:1074A00081BE0000036990F85E2010B5C3F80C257A
:1074B000036990F85D20C3F8142590F861200369F2
:1074C000012A01BF90F85F40C3F81045036990F8A6
:1074D000604006BFC3F8084503690022B1F5966F06
:1074E000C3F86C2569D9B1F5166F69D9B1F5965F06
:1074F00069D9B1F5165F68D9B1F5615F67D9B1F5A2
:10750000964F66D9B1F5E14F65D9B1F5164F64D9FB
:10751000B1F5614F64D9B1F5963F64D9B1F5E13F5A
:1075200063D9B1F5613F63D9364B994263D9B1F55F
:10753000E12F63D9B1F5612F94BF4FF070634FF025
:1075400080530269C2F8243503690422C3F8002578
:1075500001690023C1F808310169C1F81C310169D2
:1075600001230B6001698B600169C1F8042390F964
:107570005C20510902F01F0293406031224A42F818
:10758000213090F95C30002BBDBF03F00F0302F6F1
:10759000FC32D2189B18B5BF60236022137683F8A3
:1075A000002390F95C300122590903F01F0302FA0D
:1075B00003F3154A42F8213010BD4FF49E23C0E773
:1075C0004FF41D23BDE7114BBBE7114BB9E7114B3E
:1075D000B7E7114BB5E7114BB3E74FF41D03B0E725
:1075E0004FF46B03ADE70E4BABE74FF0EB73A8E73F
:1075F0004FF06C73A5E74FF08063A2E74FF0E863AC
:107600009FE700BF90D0030000E100E000B013004E
:107610000050270000F03A0000A04E0000C07500A6
:1076200000903A012DE9F0411E4600254FF47A738F
:10763000C0E901530D4B044640F8143B17468846F9
:10764000FFF798FD0A4AC4F8108084F85C7052F87D
:10765000263084F85D309DF8183052F8233084F8D5
:107660005E3084F861502046BDE8F08110C700000C
:107670007CC6000010B50369D3F8082104464AB15E
:10768000D3F818151430C9B2FFF77DFD2369002225
:10769000C3F8082110BD00000148FFF7EBBF00BF91
:1076A000EC79012007B5212300930222222303490C
:1076B0000348FFF7B7FF03B05DF804FB002000406C
:1076C000EC79012008B102F08FBD70470A4B1968B0
:1076D0000A4B30B5D3F804050C060D0A44EA000243
:1076E0004FF47A712B46A2FB014501FB0355E00BD9
:1076F00040EA454030BD00BF507A012000100140F3
:1077000038B5044648B1FFF7E1FF054600F01AF826
:10771000FFF7DCFF401BA042F8D338BD074B002227
:10772000C3F8042182B0D3F80431054A0193019BC8
:1077300013680133DBB2136002B0704700100140E0
:10774000507A01207047704708B500F05FF8FFF7E6
:10775000FAFF0120FFF7D4FFFFF712FA034CFFF7FF
:1077600021FA002CFBD0AFF30080F8E70000000006
:10777000134B53F8203010B503F01F03114C0120B8
:10778000002900FA03F010492368B3FBF1F3014626
:1077900002FB03F34FF00A02B3FBF2F314BF0246FD
:1077A00000220A4800F014F842F2107358434FF4D4
:1077B0007A722368B3FBF2F3B0FBF3F010BD00BFA5
:1077C0007CC600003000002040420F001005005031
:1077D00030B504680C40944206D1013B002BF8D12F
:1077E00012E0013B002B0FD004680C409442F8D10A
:1077F000002405680D40954204D101349C42F8D123
:10780000002002E0201C00E0181C30BD0D4BE022DF
:1078100083F811234FF40032C3F880211A604FF02F
:1078200080430122C3F818259A6003F588330021AC
:10783000C3F808150221C3F80413C3F844131A60EF
:10784000704700BF00E100E0014B1860704700BFC7
:1078500048000020222837B50CD84B4B53F8203075
:10786000052B00F0828007D8032B12D07BD8022B87
:1078700000F08180002074E01D2B78D003D81C2BF1
:10788000F8D1052206E01E2B73D01F2BF2D108225F
:1078900000E002223D4B196808296EDD0A296FDDE0
:1078A0000D29B5BF0C240E24022303233848C0F849
:1078B000F0350123C0F8003500200546030103F12F
:1078C000804303F5E04301300828C3F81455C3F89A
:1078D0001055F3D12F4B18682F4B1B6800021B0368
:1078E00003F4805300F4E0601843294BC3F81805F3
:1078F000C3F81425C3F810250DF10602C3F82C2691
:107900000122C3F830261A60D3F80021002AFBD0E8
:107910000022C3F8002101225A601D4B1A46D3F8F9
:1079200004010028FBD00020C3F804010120986066
:10793000D2F81431002BFBD00023C2F81431BDF96A
:1079400006209A42124AB8BFADF80630A142C2F8EA
:107950000035BDF9060004D035BF611A091BC840C7
:10796000884003B030BD032294E7042292E7062248
:1079700090E707228EE701228CE70824002395E791
:107980000A24012392E700BF7CC6000040000020CB
:1079900000700040440000205C7A0120222830B5AD
:1079A0003CD8224B53F82000214B00221D4653F8AF
:1079B0002240B4F1FF3F32D11E4C45F822006FEA5D
:1079C00041411D4D1D4B246853F822306FEA51414F
:1079D00025F81210012101FA04F4C3F86005013CF6
:1079E000C3F8640505EB4202C3F86805C3F86C05EB
:1079F0000020C3F80015C3F80C05C3F80405C3F84C
:107A00000845C3F81405C3F81005C3F82025C3F8CA
:107A10002415C3F82815C3F82C05996030BD84429D
:107A2000CAD00132032AC2D1F8E700BF7CC60000E9
:107A30003400002048000020547A012038C700009C
:107A4000222815D8114B124A53F8203013F0200F7A
:107A500008BF4FF0A04203F01F03032908D8DFE856
:107A600001F00210080C03F5E073002142F8231026
:107A7000704703F5E0730C21F8E703F5E073042188
:107A8000F4E703F5E0730321F0E700BF7CC60000D4
:107A900000030050222813D80A4B53F820000A4B49
:107AA00010F0200F4FF0010200F01F0008BF4FF050
:107AB000A043824011B9C3F80C257047C3F80825CC
:107AC000704700BF7CC6000000030050222810D879
:107AD000094B0A4A53F8203013F0200F08BF4FF02B
:107AE000A04203F01F03D2F81005D84000F00100B7
:107AF00070470020704700BF7CC6000000030050A4
:107B00002DE9F04106460D4601EB02080C464445BE
:107B1000A4EB050707D0336814F8011B1B68304637
:107B200098470028F3D13846BDE8F0812DE9F041AF
:107B3000C1F30A57A7F2FF35132D82B002460B4658
:107B40000C464FEAD178064633DC002D4EDB3B492C
:107B5000294103EA0100104326D049080B4052EAAC
:107B600003060CD04FF48023132D24EA010143FABD
:107B700005F444EA01040CBF4FF0004600263049EA
:107B800001EBC8082346D8E900453246204629467D
:107B900001F03EFBCDE9000122462B46DDE9000164
:107BA00001F034FB02460B461046194602B0BDE810
:107BB000F081332D07DDB5F5806FF5D101F028FB9D
:107BC00002460B46F0E7A7F213474FF0FF31F940AA
:107BD0000842E9D049080842D1D04FF0804320EA5A
:107BE000010143FA07F741EA0706C8E721F000411F
:107BF0000143D9D0C3F3130101434E42104D0E434C
:107C0000360B05EBC8055C0C06F40023D5E90067CC
:107C1000640443EA04010B463046394601F0F8FAA1
:107C2000CDE9000132463B46DDE9000101F0EEFA04
:107C300021F00041024641EAC873B5E7FFFF0F009B
:107C400048C70000F8B5C1F30A57A7F2FF35132D56
:107C50000A460B46044611DC002D2ADB8C461F49E0
:107C600029410A422BD04FF400232B41634423EADD
:107C700001030026344619462046F8BD332D05DDA4
:107C8000B5F5806F1ED011462046F8BDA7F2134708
:107C90004FF0FF3121FA07F73842F4D00122C5F145
:107CA000330502FA05F5461928BF9B1826EA070690
:107CB000E0E7013501F0004309D00026DAE70028AB
:107CC000D1D1E0E7024601F0A3FA0446DCE743F035
:107CD0007F5343F440130026CCE700BFFFFF0F00A3
:107CE00030B51F4A21F00043934287B01BDD1D4A87
:107CF000934205DD02460B4601F088FA07B030BD1D
:107D000002AA00F091F800F003000128DDE9042345
:107D100011D002281BD098B1DDE9020100F064FB0C
:107D200001F10041EAE7002300930022002301F063
:107D30009FF807B030BDDDE9020100F055FBDDE73B
:107D40000124DDE90201009401F092F8D6E7012454
:107D5000DDE90201009401F08BF801F10041CDE76B
:107D6000FB21E93FFFFFEF7F2DE9F04F8BB0044689
:107D70000D4600F077FA294B93F900A0BAF1FF3FC6
:107D800006460F4612D022462B462046294601F0D1
:107D90008FFE834650B94FF000084FF0000942466D
:107DA0004B462046294601F05BFE20B93046394655
:107DB0000BB0BDE8F08F0122194BCDF820B0009236
:107DC000CDE90445CDE902450193BAF1000F17D082
:107DD00042464B464046494601F0FAFCBAF1020FD2
:107DE000CDE906010ED101F0BFFE21230360089BFF
:107DF00073B9DDE90667304639460BB0BDE8F08F50
:107E0000CDE90689684601F073F90028EFD1EAE769
:107E100001F0AAFE089B0360EBE700BF4C000020C6
:107E200058C70000000000002DE9F04FC84E21F0B7
:107E30000047B7428FB00B4640F38F809246C54A49
:107E400097420C4626DC0029B7A3D3E9002340F370
:107E50008F8001F0DBF9C04B9F4204460D4600F0D5
:107E60004681B3A3D3E9002301F0D0F902460B46C3
:107E7000CAE900232046294601F0C8F9ACA3D3E99A
:107E8000002301F0C3F90125CAE9020128460FB019
:107E9000BDE8F08FB14A974240F38980B04A9742DB
:107EA00000F31C813D15A5F21645A7EB05531946B5
:107EB0001F46064601F012FE01F0F6FA804689469A
:107EC00002460B4630463946CDE9088901F09EF955
:107ED0000022A44B01F052FB8946804601F0FEFDD2
:107EE00001F0E2FA02460B4606460F464046494676
:107EF000CDE90A6701F08AF900229A4B01F03EFBB6
:107F000000220023CDE90C0101F0A0FD002800F0C3
:107F10005D81002330463946002201F097FD00289C
:107F200014BF01230223904A019202212A460091A4
:107F300008A8514600F07CFB002C054614DADAF85C
:107F40000420DAF80C3002F1004203F1004345420C
:107F5000CAF80420CAF80C3006E0C2E90001002586
:107F60000024C2E90245002528460FB0BDE8F08F85
:107F700001F04EF9784B9F4204460D4600F008810F
:107F80006BA3D3E9002301F043F902460B46CAE98B
:107F900000232946204601F039F965A3D3E90023DF
:107FA00001F036F94FF0FF35CAE90201DCE701F0D4
:107FB00015F861A3D3E900238046894601F0DEFA73
:107FC00000226A4B01F024F901F088FD054601F01A
:107FD0006BFA55A3D3E90023CDE9040101F0CEFAF1
:107FE00002460B464046494601F010F950A3D3E93A
:107FF0000023CDE90201DDE9040101F0BFFA1F2DE4
:108000008046894602460B46DDE9020140F3B08016
:1080100001F0FCF883460E463F15C6F30A53FB1ADF
:10802000102B40F3B08046A3D3E90023DDE904011F
:1080300001F0A4FA8046894602460B46DDE90201BA
:1080400001F0E4F802460B46DDE90201CDE9062322
:1080500001F0DCF842464B4601F0D8F83AA3D3E9E8
:10806000002380468946DDE9040101F087FA424693
:108070004B4601F0CBF80B46024680468946DDE9C7
:10808000060101F0C3F8C1F30A53FF1A312F8346EA
:108090000E4600F39D8002460B46CAE90023DDE947
:1080A0000623CDE902235A463346DDE9020101F0F9
:1080B000ADF842464B4601F0A9F8002C02460B46AB
:1080C000CAE90223BFF650AF06F1004601F10041B4
:1080D000CAE900B6CAE902016D4245E7024601F06D
:1080E00095F80025CAE90201CAE900013CE714A39A
:1080F000D3E9002301F08AF813A3D3E900230D4646
:10810000044601F083F802460B46CAE900232946DB
:10811000204601F07BF80CA3D3E9002301F076F8A8
:108120000125CAE902011FE700004054FB21F93F85
:108130003163621A61B4D03D83C8C96D305FE43FDA
:108140000000601A61B4D03D7370032E8A19A33BFE
:10815000FB21E93F7BD90240FB21F93FFB2139415B
:10816000FFFFEF7F00007041E0C700000000E03F2C
:1081700001F04CF83A4B6A1E834653F82230BB425A
:108180000E463FF449AF5A463346CAE900238AE710
:108190002BA3D3E9002301F03BF82BA3D3E9002361
:1081A0000D46044601F034F802460B46CAE90023A6
:1081B0002946204601F02AF823A3D3E9002301F041
:1081C00027F84FF0FF35CAE90201CDE60323AAE6FE
:1081D0001FA3D3E90023DDE9040101F0CFF9DDE9B4
:1081E000068906460F4602460B464046494601F0C0
:1081F0000DF802460B4640464946CDE9022301F000
:1082000005F832463B4601F001F813A3D3E90023F9
:1082100006460F46DDE9040101F0B0F932463B465F
:1082200000F0F4FF02460B4680468946DDE9020174
:1082300000F0ECFF83460E46A5E700BFAFF30080D9
:108240000000601A61B4D03D7370032E8A19A33BFD
:108250000000002E8A19A33BC14920259A837B394F
:1082600060C700005F4A8A432DE9F0410D4607468A
:1082700000F0948000290B460446064654DD0F1595
:1082800000F0A780C3F31303A7F2FF3743F4801372
:10829000F20FF80702EB43034FEA460503D5ED0F53
:1082A00005EB4303B50000267F10B44616224FF4B9
:1082B00000110CEB010098424FEAD5744FEA4505D6
:1082C00003DC1B1A00EB010C0E44013A04EB4303E0
:1082D0004FEA5101EDD11046964620244FF000425E
:1082E00009E052D05B00013C03EBD5734FEA520228
:1082F0004FEA450537D0634502EB0E01F1DD002959
:1083000001EB020E0ADBE046A3EB0C03A94288BF97
:1083100003F1FF336D1A1044C446E3E7BEF1000FCA
:10832000F1DB0CF10108EFE721F00042024329D014
:10833000002945D10146CA0A153B4905002AFAD051
:1083400012F4801001D048E030465200D40200F10F
:108350000106F9D5C6F1200401FA06F6E1401F1A1C
:1083600041EA02038EE72B4324D14408731003F142
:108370007F53F20703F5001348BF44F0004403EBBA
:10838000075127463846BDE8F081A942AAD80029FE
:1083900001EB020EC2DB98460023BBE702460B4608
:1083A00001F0ECF83A462B4600F032FF074638461B
:1083B000BDE8F081411C16BF421C01365408D5E7C8
:1083C000024600F023FF02460B4601F001FA074681
:1083D000D8E71A4621463B46B2E70E4620244FF026
:1083E000FF30BBE70000F07F2DE9F04F21F00046A1
:1083F000B6F1795F85B00C4692469B4605466BDA2E
:1084000001F06CFB002800F0E2802A462346284653
:10841000214601F0B3F874A3D3E9002380468946CE
:1084200001F0ACF872A3D3E9002300F0F1FE42465C
:108430004B4601F0A3F870A3D3E9002300F0E6FE59
:1084400042464B4601F09AF86DA3D3E9002300F0B1
:10845000DFFE42464B4601F091F86BA3D3E90023BF
:1084600000F0D4FE42464B4601F088F868A3D3E9F9
:10847000002300F0CDFE42464B4601F07FF8CDE9E7
:1084800000010022644B4046494601F077F8DDE9DF
:10849000002306460F464046494601F06FF8524613
:1084A000804689465B462846214601F067F8024629
:1084B0000B464046494600F0A9FE02460B463046B0
:1084C000394600F0A3FE02460B460020534900F057
:1084D0009DFE05B0BDE8F08F02460B4601F04EF858
:1084E00041A3D3E900238046894601F047F840A321
:1084F000D3E9002300F08CFE42464B4601F03EF8E3
:108500003DA3D3E9002300F081FE42464B4601F033
:1085100035F83BA3D3E9002300F07AFE42464B46F0
:1085200001F02CF838A3D3E9002300F06FFE424697
:108530004B4601F023F836A3D3E9002300F068FE90
:108540004B46424601F01AF8354B9E42CDE90001F8
:1085500097DD344B9E424FF000023DDCA6F5001340
:1085600000202E4916461F4600F050FECDE90201BC
:108570000022294B4046494601F000F832463B466E
:1085800000F044FEDDE9002306460F46404649461A
:1085900000F0F4FF5246804689465B462846214655
:1085A00000F0ECFF02460B464046494600F02EFE26
:1085B00002460B463046394600F028FE02460B467E
:1085C000DDE9020100F022FE05B0BDE8F08F13499D
:1085D000002005B0BDE8F08F134B144FCDE9022306
:1085E0000026C5E7AFF30080D43888BEE9FAA8BDFD
:1085F000C4B1B4BD9EEE213EAD529C804F7E923EF2
:108600009015CB19A001FA3E7751C1166CC1563FA7
:108610004C5555555555A53F0000E03F0000F03F33
:108620003233D33F0000E93F0000E73F0000D23F74
:108630002DE9F04FADF5197DBE4CA29EBE4D54F80C
:1086400026700793D41E85FB0465E417C4EBA504CC
:1086500024EAE4741D46631CA3EB8303013D02EB93
:10866000C30305937B1909940497019506460B9162
:10867000A4EB05041BD423445D1C20AF4FF000087D
:108680004FF00009DDF88CA208E05AF8240000F051
:108690000BFF0134AC42E7E8020108D0002CF4DA09
:1086A000013440464946AC42E7E80201F6D1049B5A
:1086B000002BC0F2B083079BA6F10802DB00114635
:1086C000039220AA02EB0309029301EB0308049B27
:1086D00072AA02EBC30B0DF5E07A019B002BC0F2EE
:1086E0009581039C4D460026002775E90223F4E995
:1086F000020100F043FF02460B463046394600F0C7
:1087000087FD444506460F46EFD1EAE80267DA45A1
:1087100009F10809E1D1DDE90204049920448B0044
:1087200082460BA8A3F10802C31808930CAB1344AC
:108730000A938B4698AB03EBCB03BBF1000F53E9D5
:10874000284529DD70AB03EBCB080DF13009002281
:108750007A4B2046294600F011FF01F0BFF900F0E6
:10876000A3FE0022764B06460F4600F007FF0246A6
:108770000B462046294600F049FD01F0AFF978E9A3
:10878000022349F8040B3946304600F041FD70AB36
:10879000984504460D46DAD1DDF814902046294666
:1087A0004A4600F0A9FC00224FF07F5304460D46D4
:1087B00000F0E4FE00F018FC0022624B00F0DEFE48
:1087C00002460B462046294600F020FD0D46044691
:1087D00001F084F9804600F067FE0B460246294608
:1087E000204600F013FD4B46002B06460F4640F393
:1087F000E1800BF1FF320CA9C9F1180351F82250A6
:1088000045FA03F101FA03F30CA8EB1A40F8223001
:10881000C9F11705884443FA05F5002D2CDDBBF19D
:10882000000F08F1010840F394820C9C002C40F0EA
:10883000A780BBF1010F0AD00CA9012251F8044F07
:10884000531C002C40F09E809B451A46F6D1059B98
:10885000002B0EDD012B00F09C81022B09D10BF1C6
:10886000FF320CAB0CA953F82230C3F3150341F8C7
:108870002230022D00F0AF8000220023304639461E
:1088800001F0E4F8002800F06682049B0BF1FF3948
:108890004B4510DC0BF180430CAA013B089802EB1E
:1088A0008303002253F80419834242EA0102F9D1FA
:1088B000002A40F0B580049B0CAA013B52F82330FB
:1088C000002B40F0A1800A9A012352F804190133C9
:1088D0000029FAD05B440BF101099945069349DC64
:1088E000099A079909EB020801EB0B0508F180488A
:1088F00002EB030BA39B08F1FF3803EB880870AB76
:1089000003EBC909A39B20A903EB8B0301EBC5056E
:10891000029358F8040F00F0C7FD019B002BC5E936
:10892000000105F1080B28DB083D039C0026002709
:108930000CE000BF28C90000ABAAAA2A0000703EC4
:10894000000070410000204075E80201F4E90223B4
:1089500000F014FE02460B463046394600F058FC43
:10896000544506460F46EFD1029B9845E9E8026759
:108970005D46CED1DDF818B0DCE600260027F3E72F
:10898000012300220CA9C4F180749B4541F82240C8
:108990000EDD51F8232001EB8B0001EB83036FF018
:1089A0007F4100E01A688A1A43F8042B8342F9D108
:1089B00001244CE706D10BF1FF330CAA52F82350E7
:1089C000ED152AE70022BE4B01F05EF8002840F0CA
:1089D000B981054650E732463B460020B94900F0D0
:1089E00015FC06460F46002C3FF446AF059AB549E4
:1089F000002000F081FB02460B463046394600F06D
:108A000005FC06460F4637E7012363E700260027EB
:108A1000EAE80267DA4509F108097FF45EAE7AE612
:108A20000CAB059A53F82930183ACDE90685059222
:108A30006BB909F18043013B0CA901EB830353F8A7
:108A4000041909F1FF39183A0029F8D00592059A5E
:108A50009C49002000F050FBB9F1000F04460D4680
:108A6000C0F2E0814FEAC90370AA02EB0308089341
:108A70000CAB03EB8906DFF850B208F108070436A7
:108A80004FF0000A56F8040D00F00EFD22462B466A
:108A900000F074FD5B4667E9020152462046294614
:108AA00000F06CFD0CAB9E4204460D46EAD148AB8B
:108AB00003930193CDF8149009F10103DDF81090B0
:108AC0000293C3464FF0000AB9F1000FC0F237819C
:108AD000DFF8F8815D4678A3D3E90023002600275C
:108AE000002403E0544510DCF8E80223F5E8020115
:108AF00000F044FD02460B463046394600F088FB44
:108B00000134A14506460F46ECDA019BE3E8026713
:108B10000193029B0AF1010A9A45ABF1080BD3D1EC
:108B2000A29BDDF81490032B2CD8DFE813F0E800AB
:108B3000D300D3003F00079B00200146002B40F0EC
:108B400043810D460B460B990446C1E90045039944
:108B50000246D1E9000100F059FBB9F1000F0CDD2C
:108B6000039D0124F5E90223013400F051FBA145E6
:108B7000F8DA079B002B40F037810B460B99024631
:108B8000C1E90223069B03F007000DF5197DBDE83E
:108B9000F08F0BF1FF320CAB0CA953F82230C3F36A
:108BA000160341F8223064E648AB0393B9F1000F95
:108BB00040F35581039ACDF808904FEAC90302EBC0
:108BC0000308D8E900AB0193914658E90267524681
:108BD0005B463046394600F01BFB04460D46024614
:108BE0000B463046394600F011FB52465B4600F01A
:108BF0000FFBC8E9000168E90245C145A246AB4642
:108C0000E3D1DDF80890B9F1010F40F32881019B11
:108C1000039A1344D3E9006701939A460DF5947BB8
:108C20005AE9028932463B464046494600F0F0FA8E
:108C300004460D4602460B464046494600F0E6FA19
:108C400032463B4600F0E4FACAE900016AE902450F
:108C5000D34526462F46E3D10399019C002301F119
:108C60001005083419461E46304674E9022300F008
:108C7000CFFAA5420346F6D10A460399D1E9008C02
:108C8000D1E902E90799002900F0B1800B9C23612A
:108C9000069BC4F800800CF1004009F1004102F18C
:108CA0000042606003F00700E1606261C4F808E020
:108CB0000DF5197DBDE8F08F00000040FB21F93F64
:108CC0000000E03F0000F03F0000703EF0C80000F0
:108CD00048AB0393B9F1000FFFF62DAF039F0020BF
:108CE00007EBC9060836014676E9022300F090FA40
:108CF000B742F9D1079B002B3FF423AF64E0089CF7
:108D0000039D083400222C4411461646304674E96F
:108D1000022300F07DFAA5420246F6D10B460799E0
:108D200009B103F1004319460B9B1046C3E900014A
:108D3000069B03F007000DF5197DBDE8F08F0026B6
:108D40000027E2E6BBF1000F08F101087DDD0225F6
:108D50006BE500247BE5CDE90685059D3046394667
:108D60006A4200F0C9F900223E4B06460F4600F069
:108D70008BFE00B300223C4B3046394600F0FEFB30
:108D800000F0ACFE044600F08FFB0022354B00F0F3
:108D9000F5FB0B4602463946304600F037FA00F044
:108DA0009DFE0BF101090CAB183543F82B0005951E
:108DB00043F829404BE63046394600F08FFE0CABB5
:108DC000D94643F82B0042E60B9C0B4601F10041CB
:108DD000C4E9000103990246D1E9000100F016FA46
:108DE000B9F1000F3FF7BCAE01F10041C5E61846EE
:108DF0000B9B4646744667464D461146C3E904013F
:108E0000C3E90067C3E90245069B03F007000DF5BF
:108E1000197DBDE8F08FA6F108030393079BDB00E3
:108E2000029378E4A29B032B3FF6ACAE01A252F86A
:108E300023F000BF458E0000D18C0000D18C0000D3
:108E4000A98B00000022134669E732463B4600200A
:108E5000064900F0DBF9022506460F460CE5002323
:108E60001A460AE7000070410000703E0000F03F23
:108E70002DE9F04F21F00046B6F1795F85B00C4640
:108E800090469946054604DA00F028FE002800F0D6
:108E900085802A4623462846214600F06FFB064679
:108EA0000F4602460B462846214600F067FB3EA3CC
:108EB000D3E9002382468B463046394600F05EFBFC
:108EC0003BA3D3E9002300F0A1F932463B4600F072
:108ED00055FB39A3D3E9002300F09AF932463B460B
:108EE00000F04CFB36A3D3E9002300F08FF93246A3
:108EF0003B4600F043FB34A3D3E9002300F088F99C
:108F00000E9BCDE900019BB30022334B40464946FE
:108F100000F034FBDDE90023CDE90201504659465B
:108F200000F02CFB02460B46DDE9020100F06EF971
:108F300032463B4600F022FB42464B4600F066F9C3
:108F400023A3D3E9002306460F465046594600F0B6
:108F500015FB02460B463046394600F059F90246E9
:108F60000B462846214600F051F905B0BDE8F08FC8
:108F700002460B463046394600F000FB14A3D3E905
:108F8000002300F043F952465B4600F0F7FA2A4608
:108F9000234600F03DF905B0BDE8F08F2846214694
:108FA00005B0BDE8F08F00BF7CD5CF5A3AD9E53D7A
:108FB000EB9C2B8AE6E55A3E7DFEB157E31DC73E8A
:108FC000D561C119A0012A3FA6F810111111813FE6
:108FD000495555555555C53F0000E03F21F0004328
:108FE0001946704700000000C1F30A522DE9F8430A
:108FF000A2F2FF36132E0B460D460446884607465E
:109000001DDC002E3DDB384A42FA06F901EA09026E
:10901000024319D032A3D3E9002300F0F9F800226B
:10902000002300F03BFDD0B3002D04DA4FF4801391
:1090300043FA06F6B04428EA090500272FE0332E4C
:1090400006DDB6F5806F2FD019462046BDE8F883BF
:10905000A2F213424FF0FF3929FA02F919EA000F80
:10906000F2D01FA3D3E9002300F0D2F8002200239E
:1090700000F014FD98B1002D24DB27EA09074546CE
:109080000DE017A3D3E9002300F0C2F8002200236B
:1090900000F004FD18B1002D0BDB00273D463C46D7
:1090A00029462046BDE8F883024600F0B1F80446A0
:1090B000CBE725F000430D4A1F43002F18BF15468C
:1090C0000027ECE7142E08D00123C6F1340603FA7A
:1090D00006F6371928BF9844CFE705F10108CCE719
:1090E0009C7500883CE4377EFFFF0F000000F0BF56
:1090F0000020704700000000F8B5C1F30A53044691
:109100000D460E4617460BBB21F00046034633437F
:109110001BD0354B002200F031FA344B9F420446FD
:109120000D4635DBC1F30A530E46363B3B4440F255
:10913000FE72934232DC002B11DD26F0FF4626F44E
:10914000E00646EA035520462946F8BD40F2FF7284
:109150009342EBD102460B4600F05AF8F8BD13F1EA
:10916000350F28DA4CF250339F4222462B460ADD57
:1091700019A1D1E9000100F03DF817A3D3E90023BC
:1091800000F0FCF9F8BD16A1D1E9000100F032F8B9
:1091900013A3D3E9002300F0F1F9F8BD22462B46D2
:1091A0000DA1D1E9000100F025F80BA3D3E90023BC
:1091B00000F0E4F9F8BD26F0FF4626F4E006363369
:1091C00046EA0355204629460022094B00F0D6F90D
:1091D000F8BD00BFAFF300809C7500883CE4377E8B
:1091E00059F3F8C21F6EA50100005043B03CFFFFC9
:1091F0000000903C03F0004321F0004242EA0301EA
:10920000704700BF81F0004102E000BF83F00043DF
:1092100030B54FEA41044FEA430594EA050F08BF11
:1092200090EA020F1FBF54EA000C55EA020C7FEAD5
:10923000645C7FEA655C00F0E2804FEA5454D4EB52
:109240005555B8BF6D420CDD2C4480EA020281EA1C
:10925000030382EA000083EA010180EA020281EA54
:109260000303362D88BF30BD11F0004F4FEA0131A6
:109270004FF4801C4CEA113102D0404261EB4101B5
:1092800013F0004F4FEA03334CEA133302D052423B
:1092900063EB430394EA050F00F0A780A4F10104F7
:1092A000D5F1200E0DDB02FA0EFC22FA05F2801831
:1092B00041F1000103FA0EF2801843FA05F3594117
:1092C0000EE0A5F120050EF1200E012A03FA0EFC96
:1092D00028BF4CF0020C43FA05F3C01851EBE371C0
:1092E00001F0004507D54FF0000EDCF1000C7EEBDD
:1092F00000006EEB0101B1F5801F1BD3B1F5001F1B
:109300000CD349085FEA30004FEA3C0C04F1010439
:109310004FEA445212F5800F80F09A80BCF1004F62
:1093200008BF5FEA500C50F1000041EB045141EAE4
:10933000050130BD5FEA4C0C404141EB010111F4E5
:10934000801FA4F10104E9D191F0000F04BF014690
:109350000020B1FA81F308BF2033A3F10B03B3F16E
:1093600020020CDA0C3208DD02F1140CC2F10C02FE
:1093700001FA0CF021FA02F10CE002F11402D8BF5C
:10938000C2F1200C01FA02F120FA0CFCDCBF41EA28
:109390000C019040E41AA2BF01EB0451294330BDF7
:1093A0006FEA04041F3C1CDA0C340EDC04F11404D4
:1093B000C4F1200220FA04F001FA02F340EA0300AB
:1093C00021FA04F345EA030130BDC4F10C04C4F1F1
:1093D000200220FA02F001FA04F340EA03002946D1
:1093E00030BD21FA04F0294630BD94F0000F83F41B
:1093F000801306BF81F480110134013D4EE77FEAFE
:10940000645C18BF7FEA655C29D094EA050F08BF49
:1094100090EA020F05D054EA000C04BF194610462A
:1094200030BD91EA030F1EBF0021002030BD5FEA6E
:10943000545C05D14000494128BF41F0004130BD96
:1094400014F580043CBF01F5801130BD01F00045EA
:1094500045F0FE4141F470014FF0000030BD7FEA5D
:10946000645C1ABF194610467FEA655C1CBF0B4658
:10947000024650EA013406BF52EA033591EA030F6F
:1094800041F4002130BD00BF90F0000F04BF002167
:10949000704730B54FF4806404F132044FF000059A
:1094A0004FF0000150E700BF90F0000F04BF002113
:1094B000704730B54FF4806404F1320410F0004579
:1094C00048BF40424FF000013EE700BF42004FEA74
:1094D000E2014FEA31014FEA02701FBF12F07F43F1
:1094E00093F07F4F81F06051704732F07F4208BFA8
:1094F000704793F07F4F04BF41F40021704730B5AF
:109500004FF4607401F0004521F000411CE700BFFA
:1095100050EA010208BF704730B54FF000050AE07D
:1095200050EA010208BF704730B511F0004502D57E
:10953000404261EB41014FF4806404F132045FEA80
:10954000915C3FF4D8AE4FF003025FEADC0C18BF29
:1095500003325FEADC0C18BF033202EBDC02C2F11B
:10956000200300FA03FC20FA02F001FA03FE40EAAD
:109570000E0021FA02F11444BDE600BF70B54FF0B1
:10958000FF0C4CF4E06C1CEA11541DBF1CEA13558F
:1095900094EA0C0F95EA0C0F00F0DEF82C4481EAF7
:1095A000030621EA4C5123EA4C5350EA013518BF17
:1095B00052EA033541F4801143F4801338D0A0FB04
:1095C00002CE4FF00005E1FB02E506F00042E0FBB1
:1095D00003E54FF00006E1FB03569CF0000F18BFB7
:1095E0004EF0010EA4F1FF04B6F5007F64F540745F
:1095F00004D25FEA4E0E6D4146EB060642EAC621F2
:1096000041EA55514FEAC52040EA5E504FEACE2E5E
:10961000B4F1FD0C88BFBCF5E06F1ED8BEF1004F61
:1096200008BF5FEA500E50F1000041EB045170BDDD
:1096300006F0004646EA010140EA020081EA030121
:10964000B4EB5C04C2BFD4EB0C0541EA045170BD1D
:1096500041F480114FF0000E013C00F3AB8014F197
:10966000360FDEBF002001F0004170BDC4F10004E0
:10967000203C35DA0C341BDC04F11404C4F1200561
:1096800000FA05F320FA04F001FA05F240EA0200BC
:1096900001F0004221F0004110EBD37021FA04F6F2
:1096A00042EB06015EEA430E08BF20EAD37070BDAC
:1096B000C4F10C04C4F1200500FA04F320FA05F00B
:1096C00001FA04F240EA020001F0004110EBD3700D
:1096D00041F100015EEA430E08BF20EAD37070BD7D
:1096E000C4F1200500FA05F24EEA020E20FA04F356
:1096F00001FA05F243EA020321FA04F001F0004105
:1097000021FA04F220EA020000EBD3705EEA430E75
:1097100008BF20EAD37070BD94F0000F0FD101F0A4
:109720000046400041EB010111F4801F08BF013CDD
:10973000F7D041EA060195F0000F18BF704703F01B
:109740000046520043EB030313F4801F08BF013DA2
:10975000F7D043EA0603704794EA0C0F0CEA13555E
:1097600018BF95EA0C0F0CD050EA410618BF52EA18
:109770004306D1D181EA030101F000414FF000001E
:1097800070BD50EA410606BF1046194652EA43062C
:1097900019D094EA0C0F02D150EA013613D195EAA0
:1097A0000C0F05D152EA03361CBF104619460AD1E8
:1097B00081EA030101F0004141F0FE4141F47001F2
:1097C0004FF0000070BD41F0FE4141F4780170BDE2
:1097D00070B54FF0FF0C4CF4E06C1CEA11541DBF47
:1097E0001CEA135594EA0C0F95EA0C0F00F0A7F849
:1097F000A4EB050481EA030E52EA03354FEA013176
:1098000000F088804FEA03334FF0805545EA131388
:1098100043EA12634FEA022245EA111545EA106550
:109820004FEA00260EF000419D4208BF964244F1E7
:10983000FD0404F5407402D25B084FEA3202B61A06
:1098400065EB03055B084FEA32024FF480104FF4DA
:10985000002CB6EB020E75EB030E22BFB61A75464E
:1098600040EA0C005B084FEA3202B6EB020E75EBE1
:10987000030E22BFB61A754640EA5C005B084FEA49
:109880003202B6EB020E75EB030E22BFB61A754616
:1098900040EA9C005B084FEA3202B6EB020E75EB21
:1098A000030E22BFB61A754640EADC0055EA060EE2
:1098B00018D04FEA051545EA16754FEA06164FEA25
:1098C000C30343EA52734FEAC2025FEA1C1CC0D1D1
:1098D00011F4801F0BD141EA00014FF000004FF05E
:1098E000004CB6E711F4801F04BF01430020B4F11F
:1098F000FD0C88BFBCF5E06F3FF6AFAEB5EB030CD7
:1099000004BFB6EB020C5FEA500C50F1000041EBD3
:10991000045170BD0EF0004E4EEA113114EB5C04A0
:10992000C2BFD4EB0C0541EA045170BD41F4801173
:109930004FF0000E013C90E645EA060E8DE60CEA7B
:10994000135594EA0C0F08BF95EA0C0F3FF43BAF98
:1099500094EA0C0F0AD150EA01347FF434AF95EA4F
:109960000C0F7FF425AF104619462CE795EA0C0F33
:1099700006D152EA03353FF4FDAE1046194622E700
:1099800050EA410618BF52EA43067FF4C5AE50EADA
:1099900041047FF40DAF52EA43057FF4EBAE12E7CA
:1099A0004FF0FF3C06E000BF4FF0010C02E000BFAB
:1099B0004FF0010C4DF804CD4FEA410C7FEA6C5C8E
:1099C0004FEA430C18BF7FEA6C5C1BD001B050EA31
:1099D000410C0CBF52EA430C91EA030F02BF90EA1C
:1099E000020F0020704710F1000F91EA030F58BFDB
:1099F000994208BF90422CBFD8176FEAE37040F03D
:109A0000010070474FEA410C7FEA6C5C02D150EADA
:109A1000013C07D14FEA430C7FEA6C5CD6D152EA95
:109A2000033CD3D05DF8040B704700BF844610465A
:109A300062468C461946634600E000BF01B5FFF759
:109A4000B7FF002848BF10F1000F01BD4DF808ED29
:109A5000FFF7F4FF0CBF012000205DF808FB00BFFA
:109A60004DF808EDFFF7EAFF34BF012000205DF854
:109A700008FB00BF4DF808EDFFF7E0FF94BF0120A1
:109A800000205DF808FB00BF4DF808EDFFF7CEFFA2
:109A900094BF012000205DF808FB00BF4DF808EDE1
:109AA000FFF7C4FF34BF012000205DF808FB00BFB2
:109AB0004FEA410C7FEA6C5C02D150EA013C0AD1CA
:109AC0004FEA430C7FEA6C5C02D152EA033C02D1BC
:109AD0004FF0000070474FF0010070474FEA41021D
:109AE00012F5001215D211D56FF47873B3EB6252F0
:109AF00012D94FEAC12343F0004343EA505311F017
:109B0000004F23FA02F018BF404270474FF00000A8
:109B1000704750EA013005D111F0004008BF6FF0E6
:109B2000004070474FF00000704700BF1FB51C4653
:109B3000094B1B680546D86852B1084B0091CDE926
:109B4000013207492B46224600F028F800F0B8FD04
:109B5000044B1A46F2E700BF5000002038C900004D
:109B600045C900009FB70000014B1868704700BF4F
:109B70005000002008B5074B044613B10021AFF395
:109B80000080054B1868836A03B19847204601F0AE
:109B900071FB00BF0000000074C900000EB403B5E3
:109BA000014603AB054853F8042B0068019300F00D
:109BB0007FF802B05DF804EB03B07047500000205E
:109BC00070B50D4E0D4CA41BA4100025A54209D163
:109BD0000B4E0C4C01F050FBA41BA4100025A54219
:109BE00005D170BD56F8253098470135EEE756F897
:109BF000253098470135F2E720020020200200209E
:109C0000200200203002002010B5431E0A44914279
:109C100000D110BD11F8014B03F8014FF7E788425E
:109C200010B501EB020307D8421E99420AD011F881
:109C3000014B02F8014FF8E78342F5D98118D21A97
:109C4000D34200D110BD13F8014D01F8014DF7E7E3
:109C500002440346934200D1704703F8011BF9E721
:109C60009368013B002B10B4936007DA9469A34218
:109C700001DB0A2902D110BC00F062BC1368581C39
:109C800010601970084610BC7047F8B506460F46BC
:109C90001446D518AC4201D1002007E03A4614F82A
:109CA000011B3046FFF7DCFF431CF3D1F8BD000079
:109CB0002DE9F04F9DB00C4617460393064618B1A8
:109CC00083690BB900F0F4FD7B4B9C4257D174685B
:109CD000A38918075DD52369002B5AD00023099367
:109CE00020238DF8293030238DF82A304FF0010BD6
:109CF000B846454615F8013B0BB1252B54D1B8EBBE
:109D0000070A0BD053463A4621463046FFF7BDFFBF
:109D1000013000F0C280099B5344099398F8003049
:109D2000002B00F0BA8000234FF0FF32CDE905236D
:109D3000049307938DF853301A93A846052218F818
:109D4000011B5E4800F0C4FE049B78BBD90644BFEB
:109D500020228DF853201A0744BF2B228DF8532060
:109D60002A782A2A2AD0079AA84600200A2541469E
:109D700011F8013B303B092B69D960B324E0504B0B
:109D80009C4201D1B468A3E74E4B9C4208BFF468E3
:109D90009EE72146304600F025FC00289ED04FF07B
:109DA000FF301DB0BDE8F08FA846A2E7434A801AF5
:109DB0000BFA00F0184304904546BEE7039A111DC4
:109DC00012680391002A01DB079204E0524243F03B
:109DD00002030792049398F800302E2B0ED198F8C6
:109DE00001302A2B38D1039B1A1D1B680392002BCC
:109DF000B8BF4FF0FF3308F102080593324D98F8D1
:109E000000100322284600F063FE40B14023401BAF
:109E100003FA00F0049B034308F10108049398F847
:109E200000102A488DF82810062208F1010700F0DA
:109E30004FFE002837D0264B1BBB039B073323F074
:109E4000070308330393099B4B44099350E705FB31
:109E50000232012088468AE7002308F101080593B1
:109E600019460A25404610F8012B303A092A03D931
:109E7000002BC3D00591C1E705FB012101238046DA
:109E8000F0E703AB00932246124B04A93046AFF330
:109E90000080B0F1FF3F8146D5D1A3895B063FF535
:109EA0007EAF09987DE703AB00932246094B04A9D6
:109EB000304600F087F8ECE7CCC9000078C9000014
:109EC000ECC90000ACC900007EC9000082C90000D6
:109ED000000000008B9C00002DE9F04791461F46D2
:109EE0008A680B69DDF820809342B8BF1346C9F831
:109EF000003091F8432006460C4612B10133C9F8F0
:109F000000302368990642BFD9F800300233C9F8FF
:109F10000030256815F0060507D104F1190AE36839
:109F2000D9F800209B1AAB4228DC94F84330226811
:109F3000003318BF012392062DD404F143023946A1
:109F40003046C047013020D02368E568D9F80020AA
:109F500003F00603042B08BFAD1AA36822690CBFE7
:109F600025EAE57500259342C4BF9B1AED184FF012
:109F700000091A344D451AD1002008E00123524649
:109F800039463046C047013003D14FF0FF30BDE8BD
:109F9000F0870135C3E7E1185A1C302081F84300EF
:109FA000224494F8451082F843100233C5E7012398
:109FB000224639463046C0470130E6D009F1010952
:109FC000D8E700002DE9F04301F1430C0C46097E6F
:109FD00085B06E291746064698460C9A00F0B38065
:109FE00022D8632936D00AD8002900F0B980582930
:109FF00000F0838004F1420584F8421032E06429C5
:10A0000001D06929F6D120681368050603F104011F
:10A010002AD51B681160002B03DA2D225B4284F8DD
:10A0200043206F480A2239E0732900F09D8008D848
:10A030006F2920D07029DDD1236843F020032360ED
:10A0400003E0752917D07829D4D1782384F84530D6
:10A05000644855E01368191D1B68116004F142053E
:10A0600084F8423001238CE01B68116010F0400F2F
:10A0700018BF1BB2CFE713682568181D10602806AB
:10A0800001D51B6802E06806FBD51B8854486F2980
:10A0900014BF0A220822002184F843106568A560D5
:10A0A000002DC0F29580216821F004012160002B71
:10A0B0003DD1002D40F08E806546082A0BD12368E3
:10A0C000DB0708D5236962689A42DEBF302305F8B2
:10A0D000013C05F1FF35ACEB05032361CDF80080B1
:10A0E0003B4603AA21463046FFF7F6FE01304DD12C
:10A0F0004FF0FF3005B0BDE8F083394884F84510D3
:10A10000136821681D1D1B6815600A060BD5CA0758
:10A1100044BF41F0200121601BB9226822F02002D7
:10A1200022601022B7E74D0648BF9BB2EFE76546B5
:10A13000B3FBF2F102FB1133C35C05F8013D0B46A2
:10A140000029F5D1B9E7136825686169181D106009
:10A1500028061B6801D5196002E06A06FBD5198044
:10A16000002323616546B9E71368191D11601D6856
:10A1700062680021284600F0ABFC08B1401B60601B
:10A1800063682361002384F84330A7E723692A46E4
:10A1900039463046C0470130AAD023689B0713D404
:10A1A000E068039B9842B8BF1846A3E701234A46DC
:10A1B00039463046C04701309AD00135E368039AEA
:10A1C0009B1AAB42F2DCEBE7002504F11909F5E735
:10A1D000002BACD1037884F8423004F142056CE7DF
:10A1E00089C900009AC9000038B50D4B1C68A36BE3
:10A1F00005467BB9182000F04DFC0A4A0A4BA063C3
:10A20000C0E90023094B83600B23838101220023D3
:10A21000C0E90423A36B00221D615A6138BD00BF51
:10A22000500000200E33CDAB34126DE6ECDE05009D
:10A2300038B5134B1C68A36B7BB9182000F02AFCBF
:10A24000104A114BA063C0E90023104B83600B231D
:10A25000838101220023C0E90423A16B0C480A6911
:10A260004B690C4C504304FB0300A2FB0423034442
:10A27000541C43F10005C1E9044525F0004038BDF8
:10A28000500000200E33CDAB34126DE6ECDE05003D
:10A290002DF451582D7F954C0CB430B5174B0C1E36
:10A2A0009DB01D6808DA8B232B604FF0FF301DB086
:10A2B000BDE8304002B070474FF40273ADF814307F
:10A2C00014BF04F1FF332346049307934FF6FF7343
:10A2D00002900690ADF81630209A21AB02A92846CC
:10A2E000019300F06DFD431CBCBF8B232B60002C41
:10A2F000DDD0029B00221A70D9E700BF5000002079
:10A300000EB400B59CB01DAB029006906FF00041FA
:10A31000094807910491094953F8042B05910068F5
:10A32000019302A900F04CFD029B00221A701CB0A0
:10A330005DF804EB03B07047500000200802FFFFF7
:10A3400010B503461A785C1C3AB9013B11F8012B91
:10A3500003F8012F002AF9D110BD2346F2E7C9B254
:10A36000034610F8012B1AB18A42F9D118467047FA
:10A37000002918BF0023F9E710F8012B11F8013B61
:10A38000012A28BF9A42F7D0D01A7047034613F823
:10A39000012B002AFBD1181A0138704710B56AB199
:10A3A0000139841810F8013B11F8012F934203D1B1
:10A3B000A04201D0002BF5D1981A10BD1046FCE741
:10A3C00070B50139044602B970BD234611F8015F2A
:10A3D00003F8015B561E2DB91444A342F4D003F8D0
:10A3E000015BFAE71C463246EDE7F0B503787BB136
:10A3F000044623782046661C7BB14A1E631E12F871
:10A40000015F4DB113F8017FAF423446F7D0F0E75A
:10A410000B78002B18BF0020F0BD1846FCE72DE993
:10A42000F0478046894692461E460F463D460898AC
:10A4300015F8014B00F0C6FA2044437813F00803E6
:10A4400032D12D2C32D17C78BD1C0122002E5DD062
:10A45000102E09D1302C07D12B7803F0DF03582BB5
:10A460004FD16C7810260235002A14BF4FF00041FE
:10A470006FF000410027B1FBF6FC384606FB1C1EBE
:10A48000A4F13003092B17D81C46A64223DD7B1C00
:10A4900007D084451CD301D1A64519DB00FB06403B
:10A4A000012715F8014BEBE72F46BFE72B2C04BF24
:10A4B000BD1C7C781A46C9E7A4F14103192B01D8C9
:10A4C000373CE2E7A4F16103192B04D8573CDCE7E1
:10A4D0004FF0FF37E5E77B1C08D12223C8F8003096
:10A4E0000846BAF1000F07D1BDE8F08702B140423B
:10A4F000BAF1000FF8D00FB105F1FF39CAF800909A
:10A50000F2E73024002EAFD10826ADE7302CA3D0DF
:10A510000A26A9E7084B37B51C68084D236A002BAB
:10A5200008BF2B46009313460A4601462046FFF714
:10A5300076FF03B030BD00BF50000020B400002003
:10A54000F8B50E461446054618B183690BB900F0FC
:10A55000AFF9214B9C422AD16C68A369A360A389FF
:10A560001A072ED5236963B323692068C01A63696B
:10A57000F6B28342374604DC2146284600F02EF925
:10A5800028BBA368013BA36023685A1C22601E708D
:10A5900063690130834204D0A389DB0719D50A2EF1
:10A5A00017D12146284600F019F990B10FE00B4B66
:10A5B0009C4201D1AC68D0E7094B9C4208BFEC68D3
:10A5C000CBE72146284600F00DF80028CCD04FF00C
:10A5D000FF373846F8BD00BFCCC90000ECC9000009
:10A5E000ACC90000324B70B51D6806460C4625B15B
:10A5F000AB6913B9284600F05BF92E4B9C420FD192
:10A600006C68B4F90C309AB215072CD4D00611D46A
:10A610000922326043F04003A3814FF0FF303EE057
:10A62000254B9C4201D1AC68EBE7244B9C4208BF10
:10A63000EC68E6E7510712D5616B41B104F14403C0
:10A64000994202D0304600F093FA00236363A38955
:10A6500023F02403A3810023636023692360A3897B
:10A6600043F00803A38123694BB9A38903F4207342
:10A67000B3F5007F03D02146304600F0CBF9A28924
:10A6800012F001030CD00023A36063695B42A36155
:10A69000236953B9B4F90C3013F08000BAD170BDFE
:10A6A000920758BF6369A360F2E70020F7E700BF95
:10A6B00050000020CCC90000ECC90000ACC900006B
:10A6C00008B5062000F0AAFC012000F0D3FD000030
:10A6D0008A892DE9F041054610070C4658D44B688D
:10A6E000002B05DC0B6C002B02DC0020BDE8F081A8
:10A6F000E66A002EF9D0002312F480522F68216AF6
:10A700002B6032D0606DA3895A0705D56368C01AE3
:10A71000636B0BB1236CC01A00230246E66A216A00
:10A720002846B047431CA38906D129681D2948D86B
:10A73000294ACA40D60744D500226260D90422695A
:10A74000226004D5421C01D12B6803B96065616B9E
:10A750002F600029C9D004F14403994202D0284651
:10A7600000F006FA00206063C0E701232846B047E6
:10A77000411CC8D12B68002BC5D01D2B01D0162B36
:10A7800001D12F60B1E7A38943F04003A381ADE776
:10A790000F69002FA9D093070E6808BF4B690F609F
:10A7A00018BF0023A6EB07088B60B8F1000F9CDDF3
:10A7B00043463A46216AA66A2846B047002806DC86
:10A7C000A38943F04003A3814FF0FF308EE7074495
:10A7D000A8EB0008E9E700BF0100402038B50B698D
:10A7E00005460C46DBB118B183690BB900F060F87F
:10A7F0000C4B9C4209D16C68B4F90C307BB12146FA
:10A800002846BDE83840FFF763BF074B9C4201D1A3
:10A81000AC68F1E7054B9C4208BFEC68ECE7002010
:10A8200038BD00BFCCC90000ECC90000ACC90000B5
:10A83000002310B50446C0E900338360818143667C
:10A84000C281C0E904338361194608225C30FFF7F6
:10A85000FFF9054B6362054BA362054BE362054BB1
:10A860002462236310BD00BF55B0000077B0000024
:10A87000AFB00000D3B00000014900F085B800BFC0
:10A88000DDA7000070B54A1E682555430E4605F148
:10A89000740100F0BBF9044640B10021C0E9001684
:10A8A0000C30A06005F16802FFF7D2F9204670BDB8
:10A8B000836910B5044633BBC0E912330365124BFC
:10A8C000124A1B688262984204BF0123836100F030
:10A8D0001FF86060204600F01BF8A060204600F0E2
:10A8E00017F80022E06004216068FFF7A1FF012251
:10A8F0000921A068FFF79CFF02221221E068FFF700
:10A9000097FF0123A36110BD74C9000079A800005E
:10A91000F8B51B4B1E68B369074613B93046FFF7FD
:10A92000C7FF4836D6E90134013B03D5336833B15C
:10A930003668F7E7B4F90C506DB16834F4E70421D8
:10A940003846FFF79FFF30600028F1D10C233B60B1
:10A9500004462046F8BD0B4B6566C4E90055A5606A
:10A96000C4E90335C4E905550822294604F15C0011
:10A97000FFF76EF9C4E90D55C4E91255E9E700BFC8
:10A9800074C900000100FFFF2DE9F84380468946A5
:10A9900000F14804002614B93046BDE8F883D4E934
:10A9A0000175013F01D52468F5E7AB89012B07D973
:10A9B000B5F90E30013303D029464046C847064357
:10A9C0006835EEE7D0F8EC00704770B50E46B1F987
:10A9D0000E10002996B014461D4607DA00232B609E
:10A9E000B3891A0610D44FF480630EE06A4600F073
:10A9F000A3FB0028F2DB019A02F47042A2F5005397
:10AA00005A425A412A60EEE740230020236016B0E4
:10AA100070BD00008B8973B59D0706460C4607D5AF
:10AA200004F14703236023610123636102B070BD19
:10AA300001AB6A46FFF7C9FF00990546304600F0B2
:10AA4000E5F848B9B4F90C309A05EFD423F00303C4
:10AA500043F00203A381E3E70D4BB362A3892060B7
:10AA600043F08003A381009B6361019B20615BB184
:10AA7000B4F90E10304600F071FB28B1A38923F021
:10AA8000030343F00103A381A3891D43A581CDE7FF
:10AA900079A80000024B0146186800F0B7B800BF63
:10AAA0005000002082B001B901A942B14BB1137826
:10AAB0000B601278101C18BF012002B070471046BE
:10AAC000FBE76FF00100F8E7000000000000000065
:10AAD00001F0FF01102A2BDB10F0070F08D010F84F
:10AAE000013B013A8B422DD010F0070F42B3F6D153
:10AAF000F0B441EA012141EA014122F007047FF06C
:10AB000000070023F0E80256083C85EA010586EAC2
:10AB1000010685FA47F5A3FA87F586FA47F6A5FAFE
:10AB200087F68EB9EED1F0BC01F0FF0102F007020A
:10AB300032B110F8013B013A83EA010313B1F8D1B5
:10AB40000020704701387047002D06BF3546033896
:10AB5000073815F0010F07D1013015F4807F02BFCF
:10AB6000013015F4C03F0130F0BC0138704700BF20
:10AB700038B50546002945D051F8043C0C1F002B80
:10AB8000B8BFE41800F00CFB1F4A1368104633B935
:10AB9000636014602846BDE8384000F002BBA34261
:10ABA0000CD921686218934204BF1A685B6863601D
:10ABB00004BF521822600460ECE713465A680AB1D9
:10ABC000A242FAD919685818A0420BD12068014452
:10ABD000581882421960DDD1106852685A600144E9
:10ABE0001960D7E702D90C232B60D3E7206821181E
:10ABF0008A4204BF11685268626004BF091821606C
:10AC00005C60C7E738BD00BF607A012070B5CD1C1D
:10AC100025F0030508350C2D38BF0C25002D064600
:10AC200001DBA94203D90C233360002070BD00F082
:10AC3000B7FA214A1468214691B9204C23681BB900
:10AC4000304600F0B3F920602946304600F0AEF9F6
:10AC5000431C24D10C233360304600F0A2FAE4E711
:10AC60000B685B1B18D40B2B0FD90B60CD50CC1885
:10AC7000304600F096FA04F10B00231D20F0070087
:10AC8000C31AD3D05A42E250D0E78C424B6816BF69
:10AC9000636013600C46EBE70C464968CCE7C41CC4
:10ACA00024F00304A04205D0211A304600F07EF9BA
:10ACB0000130CFD02560DBE7607A0120647A012083
:10ACC000F8B5074614460E4621B91146BDE8F840CE
:10ACD000FFF79CBF22B9FFF74BFF25462846F8BD7A
:10ACE00000F060FAA0420FD221463846FFF78EFFEF
:10ACF00005460028F2D031462246FEF785FF314650
:10AD00003846FFF735FFE9E73546E7E72DE9F04735
:10AD10008E689E4282460C469046994637D88A896C
:10AD200012F4906F31D0256809696F1A65690223A2
:10AD300005EB450595FBF3F509F101033B449D4205
:10AD400038BF1D46530530D52946FFF75FFF06463D
:10AD500050B90C23CAF80030A38943F04003A38103
:10AD60004FF0FF30BDE8F0873A462169FEF74CFF0F
:10AD7000A38923F4906343F08003A3812661656176
:10AD80003E44ED1B2660A5604E464E4500D94E461A
:10AD9000324641462068FEF742FFA3689B1BA36032
:10ADA00023681E4426600020DCE72A46FFF788FF60
:10ADB00006460028E2D121695046FFF7D9FEC8E7D0
:10ADC0002DE9F04F9DB0804603938B891D060C46FC
:10ADD00016460FD50B696BB94021FFF717FF2060AE
:10ADE000206128B90C23C8F800304FF0FF30C7E0CD
:10ADF000402363610023099320238DF829303023F9
:10AE00008DF82A304FF0010B37463D4615F8013BCF
:10AE10000BB1252B3ED1B7EB060A0BD05346324679
:10AE200021464046FFF772FF013000F0A480099BE5
:10AE3000534409933B78002B00F09D8000234FF092
:10AE4000FF32CDE90523049307938DF853301A930D
:10AE50002F46052217F8011B4F48FFF739FE049BC8
:10AE6000D0B9D90644BF20228DF853201A0744BF19
:10AE70002B228DF853202A782A2A15D0079A2F469C
:10AE800000200A25394611F8013B303B092B4DD9EA
:10AE9000B8B10FE02F46B8E73F4A801A0BFA00F02E
:10AEA000184304903D46D3E7039A111D126803919D
:10AEB000002A01DB079204E0524243F002030792AA
:10AEC00004933B782E2B0CD17B782A2B33D1039B18
:10AED0001A1D1B680392002BB8BF4FF0FF330237D7
:10AEE00005932E4D397803222846FFF7F1FD38B13E
:10AEF0004023401B03FA00F0049B034301370493F3
:10AF0000397827488DF8281006227E1CFFF7E0FDCF
:10AF1000002838D0234B13BB039B073323F00703D0
:10AF200008330393099B4B4409936DE705FB0232F9
:10AF300001200F46A6E700230137059319460A258D
:10AF4000384610F8012B303A092A03D9002BC8D013
:10AF50000591C6E705FB012101230746F0E703AB96
:10AF600000932246104B04A94046AFF30080B0F195
:10AF7000FF3F8146D6D1A3895B063FF536AF0998DE
:10AF80001DB0BDE8F08F03AB00932246064B04A929
:10AF90004046FFF717F8EAE778C900007EC90000CD
:10AFA00082C90000000000000DAD000038B5064C5D
:10AFB000002305460846236000F046F9431C02D1F1
:10AFC000236803B12B6038BDF48D01201F2938B5EB
:10AFD00004460D4604D9162303604FF0FF3038BDF8
:10AFE000426C12B152F821304BB9204600F030F8D3
:10AFF0002A4601462046BDE8384000F017B8012B2C
:10B000000AD0591C03D1162303600120E7E700246E
:10B0100042F82540284698470020E0E7024B0146C9
:10B020001868FFF7D3BF00BF5000002038B5074CA9
:10B030000023054608461146236000F0EDF8431C46
:10B0400002D1236803B12B6038BD00BFF48D01200D
:10B0500000F0D2B810B50C46B1F90E1000F0AAF805
:10B060000028ABBF636DA3891B1823F48053ACBFCA
:10B070006365A38110BD2DE9F0411F468B89DB0577
:10B0800005460C46164605D502230022B1F90E10DE
:10B0900000F074F8A389B4F90E1023F48053A3814F
:10B0A00032463B462846BDE8F04100F023B810B5D3
:10B0B0000C46B1F90E1000F061F8431CA38915BFCE
:10B0C000606523F4805343F48053A38118BFA381A8
:10B0D00010BDB1F90E1000F01FB849B1FF2A85BFAD
:10B0E0008A2303600A704FF0FF3098BF0120704739
:10B0F0000846704738B5074C0546084611460022F9
:10B1000022601A4600F0AEF8431C02D1236803B156
:10B110002B6038BDF48D012038B5064C0023054660
:10B120000846236000F058F8431C02D1236803B19D
:10B130002B6038BDF48D012038B5074C002305463F
:10B1400008461146236000F04FF8431C02D12368E3
:10B1500003B12B6038BD00BFF48D012038B5064C1B
:10B16000002305460846236000F04EF8431C02D138
:10B17000236803B12B6038BDF48D012038B5074C2E
:10B18000054608461146002222601A4600F04CF897
:10B19000431C02D1236803B12B6038BDF48D01201C
:10B1A0007047704751F8043C181F002BBCBF0B5868
:10B1B000C018704738B5074C0546084611460022AE
:10B1C00022601A4600F038F8431C02D1236803B10C
:10B1D0002B6038BDF48D0120024B58221A604FF0CD
:10B1E000FF307047F48D0120024B58221A604FF057
:10B1F000FF307047F48D0120024B58221A604FF047
:10B20000FF307047F48D0120024B58221A60002055
:10B21000704700BFF48D0120024B58221A604FF096
:10B22000FF307047F48D0120024B58221A604FF016
:10B23000FF307047F48D0120024B58221A604FF006
:10B24000FF307047F48D0120044A05491368002B34
:10B2500008BF0B461844106018467047687A0120F2
:10B26000F88D0120024B58221A604FF0FF307047D2
:10B27000F48D0120FEE700BFF8B500BFF8BC08BCA4
:10B280009E467047F8B500BFF8BC08BC9E467047A4
:10B29000646174610000000014B300001D0500002B
:10B2A0001DB300000D06000025B30000D90B0000FF
:10B2B0002CB30000E90C000031B30000330800009B
:10B2C0003CB300007706000041B30000250F0000EA
:10B2D0004DB300004F05000057B30000F10A000015
:10B2E00065B30000BF09000072B30000FB07000057
:10B2F00072616E646F6D00616C6C006C61737400E0
:10B3000066616C7365007472756500252E31357346
:10B310002E2E2E006D616B654C6973740061646440
:10B320004C6173740064656C657465006A6F696E66
:10B3300000636F707946726F6D546F0066696E645A
:10B34000006A6F696E537472696E677300756E6917
:10B35000636F6465417400756E69636F64655374EF
:10B3600072696E67006E65774279746541727261C9
:10B370007900667265654D656D6F72790000000039
:10B38000E5B300007D130000EAB30000971300004E
:10B3900025B300009B130000F0B3000081130000F0
:10B3A000FAB300009F13000003B40000A3130000D1
:10B3B0000DB40000A713000018B40000AB13000088
:10B3C00024B40000851300002DB400008F1300008A
:10B3D00037B400008913000042B40000931300004A
:10B3E00066696C65006F70656E00636C6F736500F5
:10B3F000656E644F6646696C6500726561644C6990
:10B400006E65007265616442797465730061707085
:10B41000656E644C696E6500617070656E6442793A
:10B420007465730066696C6553697A65007374614D
:10B4300072744C697374006E657874496E4C6973EC
:10B44000740073797374656D496E666F0000000057
:10B45000CC150000DC150000F0150000641600009B
:10B4600096160000C6160000F81600001A17000015
:10B47000561700008E170000DE1700001E1800008F
:10B4800086180000C4180000E41800001819000015
:10B49000581900007A190000A4190000CE19000004
:10B4A0000E1A0000861A0000441B0000B61B0000A4
:10B4B000001C0000641C0000801C00009E1C00009A
:10B4C000381D0000741D0000E41D0000121E000065
:10B4D0003A1E0000721E0000D61E00003A1F000037
:10B4E0007E1F0000C21F000032200000A2200000CA
:10B4F000EC2000003021000066210000AA2100009D
:10B50000F02100003622000088220000DE22000028
:10B510001C23000090230000C42300000A24000024
:10B520005024000096240000D024000016250000BE
:10B530005C250000B8260000A419000018190000BE
:10B54000D0250000CC150000042600002A260000AB
:10B550005E26000084260000CC150000CC150000FB
:10B56000CC150000CC1500002E2700006E2700002F
:10B57000B2270000062800002C2800007A280000CE
:10B58000A0280000D0280000CC150000CC15000039
:10B59000EE28000020290000522900008629000022
:10B5A000AA290000DE2900002C2A00004E2A0000F3
:10B5B000702A0000A22A0000D42A0000F82A000005
:10B5C0001C2B00004E2B0000722B0000CC1500003D
:10B5D000CC150000CC150000CC150000CC150000E7
:10B5E000A42B0000CA2B0000F02B0000162C00003A
:10B5F0003C2C0000702C0000A42C0000D82C000073
:10B600000C2D0000322D0000582D00008C2D000064
:10B61000CC150000CC150000CC150000CC150000A6
:10B62000CC150000CC150000CC150000CC15000096
:10B63000CC150000CC150000CC150000CC15000086
:10B64000CC150000CC150000B22D0000E22D00004A
:10B650005B2564206974656D206C6973745D0028D6
:10B6600025642062797465732900286F626A6563B6
:10B670007420747970653A202564290053746163DD
:10B680006B20756E646572666C6F7700626F6F6CAD
:10B6900065616E006E756D62657200737472696EBD
:10B6A00067006C69737400627974652061727261FD
:10B6B00079000000070000000300000015B700003B
:10B6C000FD2E00001DB70000A92F000026B70000C6
:10B6D000473000002FB70000012F000038B70000EE
:10B6E0004B30000040B7000039300000000000007F
:10B6F0000100000002000000030000000400000040
:10B700000A0000001D0000006D6963726F3A6269F3
:10B710007420763200686173546F6E6500706C61DE
:10B7200079546F6E6500686173536572766F00734C
:10B730006574536572766F00646163496E69740065
:10B74000646163577269746500474320746F6F6B5F
:10B750002025642075736563733B206672656520E0
:10B76000256420776F726473003C496E7465676569
:10B77000723E003C4C6973743E003C4F626A6563E4
:10B78000743E003C4279746541727261793E000DED
:10B790000A564D2050616E69633A2025730D0A00E8
:10B7A0006D69736300000000DDB70000613D0000BB
:10B7B000E6B70000E53C0000EAB70000313C0000BD
:10B7C000F2B70000D33B0000FCB70000653B00006F
:10B7D00008B80000673A00006E756C6C0068657808
:10B7E000546F496E740073696E006A736F6E4765BB
:10B7F00074006A736F6E436F756E74006A736F6E58
:10B8000056616C75654174006A736F6E4B65794162
:10B810007400000070B80000C13D000078B800005E
:10B82000C53D000082B80000D73D00008BB8000085
:10B83000DD3D000096B80000E33D0000A2B8000026
:10B84000E93D0000B7B80000EF3D0000CCB80000B3
:10B85000F53D0000D8B80000FB3D0000E8B800004E
:10B86000CB3D0000F4B80000D13D00006E657400CF
:10B8700068617357694669007374617274576946E9
:10B88000690073746F705769466900776966695318
:10B890007461747573006D794950416464726573A5
:10B8A000730068747470536572766572476574527C
:10B8B00065717565737400726573706F6E64546F33
:10B8C000487474705265717565737400687474702F
:10B8D000436F6E6E65637400687474704973436F70
:10B8E0006E6E65637465640068747470526571751A
:10B8F0006573740068747470526573706F6E7365ED
:10B900000000000004000000030000000A00000026
:10B910000700000006000000000000000008080802
:10B9200000080A4A4000000A5FEA5FEA0ED92ED3F7
:10B930006E19324489330C924C924D080800000075
:10B9400004880808040804848488000A448A4000A3
:10B95000048EC480000000048800000EC0000000B7
:10B9600000080001224488100C9252524C048C842E
:10B97000848E1C824C901E1EC244924C06CA525F9A
:10B98000E21FF01EC13E02448ED12E1FE2448810F9
:10B990000ED12ED12E0ED12EC48800080008000032
:10B9A000048004880244880482000EC00EC008048B
:10B9B0008244880ED126C0040ED135B36C0C925E41
:10B9C000D2521C925C925C0ED010100E1C925252FD
:10B9D0005C1ED01C901E1ED01C90100ED013712E19
:10B9E00012525ED2521C8808081C1FE242524C12AE
:10B9F00054981492101010101E113B75B13111396A
:10BA000035B3710C9252524C1C925C90100C9252B5
:10BA10004C861C925C92510ED00C825C1FE4848494
:10BA200084125252524C1131312A44113135BB71BA
:10BA300012524C9252112A4484841EC488101E0E45
:10BA4000C808080E10080482410EC242424E048A01
:10BA5000400000000000001F0804800000000ED21B
:10BA6000524F10101C925C000ED0100E02424ED2AB
:10BA70004E0C925C900E06C81C88080ED24EC24C2A
:10BA800010101C92520800080808024002424C1094
:10BA9000149814920808080806001B75B131001CA0
:10BAA000925252000C92524C001C925C90000ED2AA
:10BAB0004EC2000ED010100006C8049808080EC828
:10BAC00007001252524F0011312A4400113135BB88
:10BAD00000124C8C9200112A4498001EC4881E0645
:10BAE000C48C8486080808080818080C8818000008
:10BAF0000C83600000000000010000000200000054
:10BB00000300000004000000050000000600000023
:10BB10000700000008000000090000000A00000003
:10BB20000B0000000C0000000D0000000E000000E3
:10BB30000F000000100000001200000014000000C0
:10BB400016000000180000001A0000001C00000091
:10BB50001E0000002000000023000000260000005E
:10BB6000290000002C0000002F000000320000001F
:10BB7000360000003A0000003E00000042000000D5
:10BB8000460000004B00000050000000550000007F
:10BB90005A00000061000000680000006F00000013
:10BBA000760000007D000000840000008B00000093
:10BBB0009200000099000000A0000000A700000013
:10BBC000AE000000B5000000BC000000C300000093
:10BBD000CA000000D1000000D8000000DF00000013
:10BBE000E6000000ED000000F4000000FB00000093
:10BBF000FF00000000000000020000000400000040
:10BC000001000000030000006CBC0000153E0000B5
:10BC100077BC00008542000081BC0000D13E0000DE
:10BC20008EBC0000F140000095BC00003D410000CA
:10BC30009EBC00008D410000AABC000081400000B5
:10BC4000BBBC0000253F0000C8BC0000094000004C
:10BC5000150000001600000017000000180000008A
:10BC600019000000646973706C6179006C69676821
:10BC7000744C6576656C006D62446973706C6179B3
:10BC8000006D62446973706C61794F6666006D6225
:10BC9000506C6F74006D62556E706C6F74006D62E5
:10BCA000447261775368617065006D6253686170BA
:10BCB00065466F724C6574746572006E656F50698D
:10BCC00078656C53656E64006E656F506978656C5D
:10BCD00053657450696E004E6F7420656E6F7567A2
:10BCE0006820726F6F6D206576656E206166746581
:10BCF0007220636F6D70616374696F6E00436F6D66
:10BD000070616374656420466C61736820636F645E
:10BD1000652073746F72650A256420627974657397
:10BD2000207573656420282564252529206F6620E9
:10BD3000256400426164207265636F726420666FDF
:10BD4000756E6420647572696E6720696E697469C6
:10BD5000616C697A6174696F6E00256420256420C6
:10BD600025642028256420776F7264732900256478
:10BD7000207265636F7264732C20256420776F7264
:10BD800064732C206D617849442025642C20636FF6
:10BD90006D70616374696F6E206379636C65732085
:10BDA000256400526573746F726564202564207386
:10BDB00063726970747300537461727465640072A5
:10BDC0006164696F0000000058BE0000414B000034
:10BDD00065BE0000B54D000075BE0000494D000075
:10BDE00083BE0000154F00008EBE0000694B0000AE
:10BDF0009EBE0000F94B0000B2BE0000DD4B00000B
:10BE0000C1BE0000F1500000CDBE00006D5000002A
:10BE1000D6BE000011500000E1BE0000614F0000DE
:10BE2000ECBE0000994F0000F5BE0000C94F0000B5
:10BE3000FEBE0000794B00000DBF0000594B000012
:10BE400016BF0000894B00006E6F6E65006F74684E
:10BE5000657200706169720064697361626C655239
:10BE60006164696F006D65737361676552656365D1
:10BE700069766564007061636B65745265636569BA
:10BE80007665007061636B657453656E64007265FE
:10BE9000636569766564496E74656765720072658D
:10BEA0006365697665644D65737361676554797020
:10BEB00065007265636569766564537472696E675F
:10BEC0000073656E64496E74656765720073656EB4
:10BED00064506169720073656E64537472696E6751
:10BEE000007365744368616E6E656C0073657447BA
:10BEF000726F757000736574506F77657200736947
:10BF0000676E616C537472656E6774680064657601
:10BF10006963654944006C6173744D65737361674F
:10BF200065494400556E6B6E6F776E207072696D57
:10BF30006974697665205B25733A25735D0000009E
:10BF400000000000963007772C610EEEBA51099977
:10BF500019C46D078FF46A7035A563E9A395649ED3
:10BF60003288DB0EA4B8DC791EE9D5E088D9D297F7
:10BF70002B4CB609BD7CB17E072DB8E7911DBF9053
:10BF80006410B71DF220B06A4871B9F3DE41BE8477
:10BF90007DD4DA1AEBE4DD6D51B5D4F4C785D383D3
:10BFA00056986C13C0A86B647AF962FDECC9658A77
:10BFB0004F5C0114D96C0663633D0FFAF50D088DD3
:10BFC000C8206E3B5E10694CE44160D5727167A277
:10BFD000D1E4033C47D4044BFD850DD26BB50AA5D3
:10BFE000FAA8B5356C98B242D6C9BBDB40F9BCACF7
:10BFF000E36CD832755CDF45CF0DD6DC593DD1AB53
:10C00000AC30D9263A00DE518051D7C81661D0BF76
:10C01000B5F4B42123C4B3569995BACF0FA5BDB8D2
:10C020009EB802280888055FB2D90CC624E90BB176
:10C03000877C6F2F114C6858AB1D61C13D2D66B6D2
:10C040009041DC760671DB01BC20D2982A10D5EF36
:10C050008985B1711FB5B606A5E4BF9F33D4B8E892
:10C06000A2C9077834F9000F8EA8099618980EE136
:10C07000BB0D6A7F2D3D6D08976C6491015C63E692
:10C08000F4516B6B62616C1CD83065854E0062F2B6
:10C09000ED95066C7BA5011BC1F4088257C40FF512
:10C0A000C6D9B06550E9B712EAB8BE8B7C88B9FC36
:10C0B000DF1DDD62492DDA15F37CD38C654CD4FB92
:10C0C0005861B24DCE51B53A7400BCA3E230BBD436
:10C0D00041A5DF4AD795D83D6DC4D1A4FBF4D6D392
:10C0E0006AE96943FCD96E34468867ADD0B860DA36
:10C0F000732D0444E51D03335F4C0AAAC97C0DDD92
:10C100003C710550AA41022710100BBE86200CC9B5
:10C1100025B56857B3856F2009D466B99FE461CE11
:10C120000EF9DE5E98C9D9292298D0B0B4A8D7C735
:10C13000173DB359810DB42E3B5CBDB7AD6CBAC091
:10C140002083B8EDB6B3BF9A0CE2B6039AD2B174AD
:10C150003947D5EAAF77D29D1526DB048316DC7309
:10C16000120B63E3843B64943E6A6D0DA85A6A7AAD
:10C170000BCF0EE49DFF099327AE000AB19E077D09
:10C1800044930FF0D2A3088768F2011EFEC206692D
:10C190005D5762F7CB67658071366C19E7066B6E89
:10C1A000761BD4FEE02BD3895A7ADA10CC4ADD67AD
:10C1B0006FDFB9F9F9EFBE8E43BEB717D58EB06009
:10C1C000E8A3D6D67E93D1A1C4C2D83852F2DF4FAD
:10C1D000F167BBD16757BCA6DD06B53F4B36B24809
:10C1E000DA2B0DD84C1B0AAFF64A0336607A0441AD
:10C1F000C3EF60DF55DF67A8EF8E6E3179BE694609
:10C200008CB361CB1A8366BCA0D26F2536E268522C
:10C2100095770CCC03470BBBB91602222F26055588
:10C22000BE3BBAC5280BBDB2925AB42B046AB35CAC
:10C23000A7FFD7C231CFD0B58B9ED92C1DAEDE5B08
:10C24000B0C2649B26F263EC9CA36A750A936D02EC
:10C25000A906099C3F360EEB856707721357000548
:10C26000824ABF95147AB8E2AE2BB17B381BB60C6C
:10C270009B8ED2920DBED5E5B7EFDC7C21DFDB0BC8
:10C28000D4D2D38642E2D4F1F8B3DD686E83DA1FEC
:10C29000CD16BE815B26B9F6E177B06F7747B71848
:10C2A000E65A0888706A0FFFCA3B06665C0B0111EC
:10C2B000FF9E658F69AE62F8D3FF6B6145CF6C1648
:10C2C00078E20AA0EED20DD75483044EC2B30339EC
:10C2D000612667A7F71660D04D476949DB776E3E48
:10C2E0004A6AD1AEDC5AD6D9660BDF40F03BD8376C
:10C2F00053AEBCA9C59EBBDE7FCFB247E9FFB530C8
:10C300001CF2BDBD8AC2BACA3093B353A6A3B424EB
:10C310000536D0BA9306D7CD2957DE54BF67D92347
:10C320002E7A66B3B84A61C4021B685D942B6F2AEB
:10C3300037BE0BB4A18E0CC31BDF055A8DEF022D47
:10C34000416C6C207461736B732073746F707065D3
:10C3500064007631303300202573202573004D654D
:10C360006D6F727920636C6561726564004E6F2039
:10C3700066726565207461736B20656E74726965A1
:10C3800073000000DCC30000F5650000E9C3000095
:10C3900071600000F5C30000C5650000FBC300002C
:10C3A000D565000001C40000E565000007C4000079
:10C3B000A160000011C400003D66000019C4000027
:10C3C0009163000022C40000296100002AC400001B
:10C3D000C162000073656E736F72730061636365A1
:10C3E0006C65726174696F6E0074656D7065726101
:10C3F000747572650074696C74580074696C745952
:10C400000074696C745A00746F7563685265616476
:10C4100000693263526561640069326357726974FE
:10C42000650072656164444854006D6963726F70A1
:10C43000686F6E6500000000ACC40000BD660000BF
:10C44000BAC40000C1660000C3C40000CD6600008D
:10C45000CDC40000D1660000D6C40000D56600003F
:10C46000DBC40000D9660000E0C40000DD66000007
:10C47000ECC40000E1660000F3C40000E5660000C3
:10C48000FCC40000E966000001C50000ED66000084
:10C490000CC50000F166000016C50000C56600006E
:10C4A00020C50000C966000074667400656E616294
:10C4B0006C65446973706C61790067657457696471
:10C4C00074680067657448656967687400736574AB
:10C4D000506978656C006C696E6500726563740004
:10C4E000726F756E6465645265637400636972632C
:10C4F0006C6500747269616E676C65007465787450
:10C5000000746674546F756368656400746674546F
:10C510006F7563685800746674546F75636859006A
:10C52000746674546F756368507265737375726561
:10C53000007661727300000058C50000556B000062
:10C5400062C50000356B00006BC50000116B000078
:10C5500077C50000A36A000076617245786973743C
:10C5600073007661724E616D656400736574566127
:10C57000724E616D6564007661724E616D65466FE5
:10C5800072496E6465780057656C636F6D652074E1
:10C590006F204D6963726F426C6F636B7321007023
:10C5A0005F73706920213D204E554C4C002F726FF7
:10C5B0006F742F2E706C6174666F726D696F2F705F
:10C5C00061636B616765732F6672616D65776F720A
:10C5D0006B2D61726475696E6F6E6F726469636EE4
:10C5E000726635407372632D316636363436356285
:10C5F000633137346633363633373938396537384F
:10C6000065333862636363382F6C69627261726983
:10C6100065732F5350492F5350492E637070005348
:10C620005049436C6173733A3A535049436C617398
:10C6300073284E52465F5350495F547970652A2CD7
:10C640002075696E74385F742C2075696E74385F5C
:10C65000742C2075696E74385F7429000000000026
:10C6600000000000556D00000D6D0000436D0000DE
:10C67000496D00004F6D0000416D00000200000098
:10C6800003000000040000001F0000001C00000068
:10C690000E000000250000000B0000000A00000052
:10C6A000090000001E000000170000000C00000040
:10C6B00011000000010000000D0000002200000039
:10C6C000FFFFFFFFFFFFFFFF1A0000002000000038
:10C6D00015000000160000000F0000001800000008
:10C6E00013000000240000000000000014000000FF
:10C6F0000500000010000000080000001900000004
:10C7000006000000280000000000000000000000FB
:10C710001B740000017B0000917400009D740000F8
:10C72000977400001974000011740000A5740000D3
:10C73000357400000D74000000C00140001002407C
:10C740000020024000000000000000000000304314
:10C7500000000000000030C373717274000000001C
:10C76000FB21F93FFB2109407CD91240FB211940F4
:10C770007A6A1F407CD92240BBFD2540FB2129401D
:10C780003A462C407A6A2F405C4731407CD932408F
:10C790009C6B3440BBFD3540DB8F3740FB2139407B
:10C7A0001BB43A403A463C405AD83D407A6A3F4032
:10C7B0004C7E40405C4741406C1042407CD9424036
:10C7C0008CA243409C6B4440AC344540BBFD45408B
:10C7D000CBC64640DB8F4740EB584840FB214940E1
:10C7E00083F9A200444E6E00FC291500D1572700A2
:10C7F000DD34F50062DBC0003C99950041904300B8
:10C800006351FE00BBDEAB00B761C5003A6E240089
:10C81000D24D42004906E00009EA2E001C92D100E8
:10C82000EB1DFE0029B11C00E83EA700F535820093
:10C8300044BB2E009CE98400B4267000417E5F005A
:10C84000D6913900538339009CF439008B5F840002
:10C8500028F9BD00F81F3B00DEFF97000F98050088
:10C86000112FEF000A5A8B006D1F6D00CF7E36002E
:10C8700009CB2700464FB7009E663F002DEA5F00B8
:10C88000BA277500E5EBC7003D7BF100F7390700DB
:10C8900092528A00FB6BEA001FB15F00085D8D00B9
:10C8A000300356007BFC4600F0AB6B0020BCCF0091
:10C8B00036F49A00E3A91D005E619100081BE600B2
:10C8C00085996500A0145F008D40680080D8FF0046
:10C8D00027734D0006063100CA561500C9A873001B
:10C8E0007BE260006B8CC00000000040FB21F93F40
:10C8F000000000002D44743E000000809846F83C83
:10C900000000006051CC783B00000080831BF039B0
:10C910000000004020257A38000000802282E336A3
:10C92000000000001DF36935020000000300000054
:10C9300004000000060000002C2066756E63746918
:10C940006F6E3A2000617373657274696F6E202296
:10C95000257322206661696C65643A2066696C659E
:10C9600020222573222C206C696E65202564257396
:10C9700025730A0054000020232D302B2000686C02
:10C980004C006566674546470030313233343536F2
:10C99000373839414243444546003031323334352B
:10C9A0003637383961626364656600000000000054
:10C9B0000000000000000000000000000000000077
:10C9C0000000000000000000000000000000000067
:10C9D0000000000000000000000000000000000057
:10C9E0000000000000000000000000000000000047
:10C9F0000000000000000000000000000000000037
:10CA00000000000000000000000000004300504F44
:10CA100053495800002020202020202020202828B2
:10CA200028282820202020202020202020202020EE
:10CA3000202020202088101010101010101010102E
:10CA4000101010101004040404040404040404105E
:10CA500010101010101041414141414101010101EC
:10CA600001010101010101010101010101010101B6
:10CA700010101010101042424242424202020202C2
:10CA80000202020202020202020202020202020286
:10CA90001010101020000000000000000000000036
:10CAA0000000000000000000000000000000000086
:10CAB0000000000000000000000000000000000076
:10CAC0000000000000000000000000000000000066
:10CAD0000000000000000000000000000000000056
:10CAE0000000000000000000000000000000000046
:10CAF0000000000000000000000000000000000036
:10CB00000000000000000000000000000000000025
:0CCB100000000000000000000000000019
:08CB1C002439FF7F0100000035
:10CB2400FFFFFFFFD007000001000000E803DC0561
:10CB3400DC05DC05DC050000FFFFFFFFFFFFFFFF56
:10CB44001800000019FCFFFFFFFFFFFFFF000000BB
:10CB54000090D003FFFFFFFFFFFFFFFFFFFFFFFF7A
:10CB64000A000000010000000800000001000000AD
:10CB74005400002000000000CCC90000ECC90000F3
:10CB8400ACC900000000000000000000000000002C
:10CB94000000000000000000000000000000000091
:10CBA4000000000000000000000000000000000081
:10CBB4000000000000000000000000000000000071
:10CBC4000000000000000000000000000000000061
:10CBD400000000004300000000000000000000000E
:10CBE4000000000000000000000000000000000041
:10CBF40000000000430000000000000000000000EE
:10CC04000000000000000000000000000000000020
:10CC140000000000430000000000000000000000CD
:10CC24000000000000000000000000000000000000
:10CC340000000000430000000000000000000000AD
:10CC440000000000000000000000000000000000E0
:10CC5400000000004300000000000000000000008D
:10CC640000000000000000000000000000000000C0
:10CC7400000000004300000000000000000000006D
:10CC840000000000000000000000000000000000A0
:10CC9400000000004300000000000000000000004D
:10CCA4000000000000000000000000000000000080
:10CCB40000000000DBB00000A5AA00000000000096
:10CCC40014CA000012B300009FB700009FB7000011
:10CCD4009FB700009FB700009FB700009FB70000F8
:10CCE4009FB700009FB700009FB70000FFFFFFFF42
:10CCF400FFFFFFFFFFFFFFFFFFFF000001004153A5
:10CD0400434949000000000000000000000000004A
:10CD1400000000000000000000000000000041537B
:10CD2400434949000000000000000000000000002A
:10CD340000000000000000000000000000000000EF
:10CD440025040000D96C000035710000A5760000B0
:04CD540001040000D6
:04000003000071F197
:00000001FF
